:020000040800F2
:10000000D010002005010008F73700080929000872
:10001000F5370008350F0008916000080000000067
:10002000000000000000000000000000D9460008A9
:10003000BD1A000800000000653D0008C149000825
:100040001F010008653B00081F0100081F01000890
:100050001F0100081F0100081F0100081F01000800
:100060001F0100081F0100081F0100081F010008F0
:100070001F0100081F010008791500081F01000872
:100080001F0100081F010008410700081F010008A8
:100090001F0100081F0100081F0100081F010008C0
:1000A000314A0008114B00081F0100081F01000819
:1000B000154B0008054E0008615000081F0100089C
:1000C0001F0100081F0100081F0100081F01000890
:1000D0001F010008895B00081F0100081F010008BC
:1000E0001F0100081F0100081F010008DFF810D0E1
:1000F00000F0E8FA00480047B1710008AFF3008053
:10010000D01000200648804706480047FEE7FEE77B
:10011000FEE7FEE7FEE7FEE7FEE7FEE7FEE7FEE7B7
:10012000E1490008ED0000082DE9F0410024061B1C
:10013000254671F1000605DA01240027D0EB0700FF
:1001400067EB0101161E73F1000605DA0027D2EBFA
:100150000702012567EB030300F0D0F986460E463F
:1001600017469C46AC4204D00025D0EB050E65EB4B
:10017000010624B10020D2EB000760EB030C7046AF
:1001800031463A466346BDE8F08140EA01039B07E9
:1001900003D009E008C9121F08C0042AFAD203E0FC
:1001A00011F8013B00F8013B521EF9D2704780EA7A
:1001B000010210B502F00043400022D04A001FD0D7
:1001C000010E01EB1261C0F35600C2F3560240F477
:1001D000000042F40002A0FB022000047F39140456
:1001E00000D0401C50EA124001D44000491EC2B267
:1001F0000C0604EBD010401C4008802A02D003E01B
:10020000002010BD20F00100002900DA0020184372
:1002100010BD2DE9FE4F81EA030404F0004421F0F3
:10022000004100944FF0000B23F0004350EA01041A
:100230005ED052EA03045BD0C3F30A54C1F30A55FB
:100240002C44A4F2F3340194A0FB0254C1F3130133
:1002500041F48011C3F3130343F4801301FB024400
:1002600000FB034E840A970A44EA815447EA835705
:10027000A4FB076802958D0A05FB07854FEA932CBE
:1002800004FB0C542705029D4FEA065847EA16372F
:10029000B5EB08056EEB070C870E920E47EA811747
:1002A00042EA8312A7FB0201B6EB0B0164EB0004E8
:1002B0002B0D43EA0C335E1844EB1C50DA465146D2
:1002C000E7FB0201C5F313044FEA0B3343EA14536F
:1002D0004FEA0432019C43EA0603A4F10C040294A1
:1002E000009CCDE900B400F09FF903B0BDE8F08FA9
:1002F00000200146F9E72DE9F04D81EA030404F0FE
:10030000004B21F0004514464FF0000A23F0004155
:1003100050EA050220D054EA01021DD0C5F30A5765
:100320000246C5F31303C1F31300C1F30A5640F4A8
:10033000801543F48013A7EB0608101BD64608F27D
:10034000FD3873EB050002D308F1010801E09218B3
:100350005B41B8F1000F03DA00200146BDE8F08DE3
:1003600000204FF48011064684460EE0171B73EB05
:10037000050705D3121B63EB050306434CEA010C8A
:1003800049084FEA300092185B4150EA0107EDD16D
:1003900052EA030012D082EA040083EA050108430E
:1003A00005D0101BAB4106D20122002306E000223B
:1003B0004FF0004302E06FF0010253101AEB060009
:1003C0004CEB085110EB0A0041EB0B01BDE8F04D7E
:1003D00000F01BB970B521F0004303430CD0C1F30A
:1003E0000A550024D5EB040564EB0403D617AD1AB7
:1003F000B34102DB0020014670BD201841EB0251E1
:1004000070BDC10F80EAE0700844CA07962300213E
:1004100000F0CDB896230022114600F0C8B80EB502
:10042000C10F80EAE0700844CA07002140F233435C
:100430008DE80E000A460B4600F0F6F803B000BD4A
:100440000EB540F2334102910021CDE900110A4678
:100450000B4600F0E9F803B000BD00F0004220F0C8
:100460000040C10DC0F3160040F400007F2901DAFE
:1004700000207047962903DCC1F19601C84001E0D5
:1004800096398840002AF4D04042704770B5C1F3D5
:100490000A5201F000450024C1F3130140F2FF337A
:1004A00041F480119A4201DA002070BD40F23343DA
:1004B0009A42A2F2334203DC524200F05FF800E0BD
:1004C00090402C43F1D0404270BDC1F30A5210B5A8
:1004D000C1F3130140F2FF3341F480119A4201DA73
:1004E000002010BD40F233439A42A2F2334203DCB3
:1004F000524200F043F810BD904010BD2DE9F05F6E
:100500000546002092469B46884606468146402482
:100510001BE0284641464746224600F02FF8534646
:100520005A46C01A914110D311461846224600F08F
:1005300016F82D1A67EB01084F46224601200021CC
:1005400000F00DF817EB00094E41201EA4F1010444
:10055000DFDC484631462A464346BDE8F09F202A64
:1005600004DB203A00FA02F1002070479140C2F10A
:10057000200320FA03F3194390407047202A04DB3C
:10058000203A21FA02F00021704721FA02F3D0400C
:10059000C2F1200291400843194670470029A8BFC4
:1005A0007047401C490008BF20F00100704710B49C
:1005B000B0FA80FC00FA0CF050EA010404BF10BC51
:1005C000704749B1CCF1200421FA04F411FA0CF17E
:1005D00018BF012121430843A3EB0C01CB1D4FEAB7
:1005E00000614FEA102042BF002010BC704700EBB2
:1005F000C35010440029A4BF10BC7047401C4900E0
:1006000008BF20F0010010BC704710B5141E73F134
:10061000000408DA401C41F1000192185B411A43C2
:1006200001D120F0010010BD2DE9F04D92469B460E
:1006300011B1B1FA81F202E0B0FA80F220329046B4
:10064000FFF78DFF04460F4640EA0A0041EA0B011E
:1006500053465A46084313D0114653EA010019D0B5
:10066000C8F140025046FFF789FF05460E46504646
:1006700059464246FFF773FF084305D0012004E0C6
:1006800020463946BDE8F08D0020054346EAE07675
:100690002C4337430A986305E40AA0EB08000022C4
:1006A000FD0A44EA47540A3002D500200146E9E732
:1006B000010510196941DDE9084500196941BDE8E6
:1006C000F04DA2E7064C074D06E0E06840F001035C
:1006D00094E8070098471034AC42F6D3FFF70AFDC0
:1006E000F49100081492000870B58C1810F8015BA2
:1006F00015F0070301D110F8013B2A1106D110F8BB
:10070000012B03E010F8016B01F8016B5B1EF9D1BE
:100710002B0705D40023521E0DD401F8013BFAE744
:1007200010F8013BCB1A921C03E013F8015B01F8AF
:10073000015B521EF9D5A142D8D3002070BD000044
:1007400070B54E4C4FF490652946204600F019FADA
:10075000002864D02946204600F0A6F848490888B9
:10076000401C08800121204600F0EAFA454942F287
:100770001072B1F85000904202D2401CA1F8500013
:1007800006F0F6FE404DB5F91410B5F9120005F06B
:10079000B1FD3E4CA5F84E002080A1682046884758
:1007A000A088A5F8500003F08FF806F0E3FF384E5C
:1007B000384C3078082833D045F6AC30606042F6CB
:1007C000EF60A06042F2C400E0603348008A2080FD
:1007D000208E6080A16B2F488847208E69882F4C1F
:1007E00008444FF6FF7101EA80006886207A4FF0D6
:1007F000000540071DD501F0F1FA294949F6A2404C
:100800000880284840F21A62C188491C89B2C18018
:10081000914204D3A16821F00401A160C58070BD9C
:1008200041F2130060604FF48060A06040F61B50FE
:10083000CAE730780A281BD2DFE800F01A0616054E
:100840000A050D1A1114EAE7BDE8704005F0F6BE7E
:1008500007F086FE08E0BDE8704002F07FBD06F0BC
:100860007FFA01E007F0DEF8BDE8704007F0DAB883
:1008700000F0F8FB84F8B65070BD00000024014081
:10088000F80600203C010020600000201407002032
:10089000EF060020D0000020EC010020980200208C
:1008A000442C0140180900206FEA112101607047B3
:1008B0000029816802D041F0010101E021F001012D
:1008C000816070470029816802D041F4807101E0A5
:1008D00021F48071816070472DE9F041824E92B021
:1008E000304600F00BF90BA800F039FA01214FF463
:1008F000C06003F0EDFA00248DF831404FF4602021
:10090000CDE90D044FF4A0204FF009080B9001270A
:100910008DF83C808DF830700BA9304600F080F9DE
:10092000724D8DF831408DF830708DF83C700BA908
:10093000284600F075F901231A460F21304600F0D1
:10094000C0F9022201231146304600F0BAF9012312
:1009500003220021304600F0B4F901230422194695
:10096000304600F0AEF9012305220B21304600F09D
:10097000A8F9012306220421304600F0A2F9012340
:1009800007220821304600F09CF9012308220321A8
:10099000304600F096F9012309220A21304600F082
:1009A00090F90121304600F084F90121284600F039
:1009B00080F901231A460521304600F055F901233C
:1009C0001A460621284600F04FF90021304600F073
:1009D000CBF84FF4E041284600F0C6F8012130463C
:1009E00000F0B8F80121284600F0B4F801213046A3
:1009F00000F0A6F80121284600F0A2F801213046B7
:100A000000F09EF90121284600F09AF940F61451B1
:100A1000374804F0FCFD12208DF8400002208DF8CC
:100A200041008DF842408DF8437010A802F010FF8D
:100A300001224FF49061304600F0E8F80121304681
:100A4000FFF740FF01213046FFF732FF0121284622
:100A5000FFF72EFF304600F06EF9304600F09FF8A9
:100A60000028FAD1304600F075F9304600F082F8DF
:100A70000028FAD1284600F05EF9284600F08FF8E9
:100A80000028FAD1284600F065F9284600F072F8EF
:100A90000028FAD10121084603F0F6F9154D284641
:100AA00000F0A6FD684600F04EFE0F4801A94C304C
:100AB0000090114881E811018020CDE904404000F8
:100AC000069080000790202008904FF44050CDE918
:100AD00009046946284600F019FE0121284600F065
:100AE0007BFD12B0BDE8F0810024014000280140E8
:100AF000002C014008000240A80200200D4910B55A
:100B0000884202D1012144150AE00B49884202D1F2
:100B10000121041504E0094988420AD10121CC03CE
:100B2000204603F0E1F92046BDE81040002103F023
:100B3000DBB910BD0024014000280140003C014009
:100B40000029816802D041F4801101E021F4801174
:100B5000816070470029816802D041F4004101E0C2
:100B600021F4004181607047826822F4E0420A4328
:100B700082607047014600208968490700D501203E
:100B8000704710B50246002054680B0AC9B20C40E9
:100B90001168194202D0002C00D0012010BD01467E
:100BA00000208968090700D50120704738B5012168
:100BB0001C2003F08DF9FF20ADF8000000248DF813
:100BC000034003258DF8025069460D4801F00CFBE7
:100BD0000120ADF800008DF803408DF80250694601
:100BE000084801F001FB2320ADF800008DF8034018
:100BF0008DF802506946044801F0F6FA38BD00004D
:100C000000080140000C014000100140002A426829
:100C1000C9B201D00A4300E08A4342607047000035
:100C200010B542680E4B0C791A400B6842EA042258
:100C30001343436083680B4A1340D1E902422243C5
:100C40004C7943EA44031A438260C26A097C22F465
:100C50007002491EC9B242EA0151C16210BD0000D2
:100C6000FFFEF0FFFDF7F1FF70B5072409290AD94F
:100C7000C568A1F10A0606EB4606B440A543B34099
:100C80001D43C56007E0056901EB4106B440A5437B
:100C9000B3401D430561836BC3F30154121B921CC7
:100CA00002EB82041F22A2409343A1400B438363C3
:100CB00070BD826B491E22F4401242EA01518163E9
:100CC000704770B5072409290AD9C568A1F10A0639
:100CD00006EB4606B440A543B3401D43C56007E09C
:100CE000056901EB4106B440A543B3401D430561CE
:100CF0001F23072A09D2446B521E02EB8202934043
:100D00009C4391400C43446370BD0D2A09D2046B8F
:100D1000D21F02EB820293409C4391400C43046338
:100D200070BDC46A0D3A02EB820293409C4391402D
:100D30000C43C46270BD816841F008018160704756
:100D40000029816802D041F4A00101E021F4A00152
:100D500081607047816841F0040181607047002123
:100D60000160017141718160C160012101747047AE
:100D700070B51E4C214694F83800B1F84250062850
:100D80001ED9B4F84A10B4F84C00A1EB000202F1ED
:100D90000902122A04D8FFF753FB0022144B0AE081
:100DA000884204D2FFF74CFB0022124B03E0FFF70E
:100DB00047FB0022104BFFF72CFAFFF786FB09E0F8
:100DC00005D12846FFF73CFB0C4A0D4BF3E70D49D4
:100DD00051F82000C5EB45116063B0EB410F03D91A
:100DE000C5EB45104000606370BD00003C0400206E
:100DF00000003440000033400000354067666666FE
:100E000066E64B409C89000810B50C4C20784007E2
:100E100013D5FFF7ADFF0A49A08E08800848303887
:100E2000018821F010010180001F018841F01001AC
:100E30000180207820F00400207010BD3C040020C8
:100E400040040040F0B41448144B154A816804462D
:100E50001B782468526CCF0541F0080521F0080684
:100E60004FEA047413D5002C07DB090712D4002BBA
:100E700010D1142A0EDA856006E009070AD5002B86
:100E800008D1142A06DA8660F0BC05F06DBD002C8E
:100E9000F3DAEAE7F0BC704798020020EF06002082
:100EA0003C01002070B506464089204B204C4FF491
:100EB0008071002580B362887AB1012A0CD1E18863
:100EC000491C89B2E1803289914205D36580E58071
:100ED000FF2801D0401E708170BD7088228890422A
:100EE00001D9012200E00022184601F006FA7088BC
:100EF000B18801442088401C80B220808142EBD818
:100F00002580A088401C80B2A080F1888842E3D36D
:100F100001206080A58070BDFFE70022184601F027
:100F2000ECF9A580E58025806580F4E7000C0140A0
:100F3000AC050020FEE70000FCB505464FF6FF7645
:100F400000200C46ADF8006048F205078DF804005B
:100F500020E000BF15F8010B8DF8040001A9084638
:100F600002F0DAF8BDF800009DF8041080EA0120D4
:100F7000ADF800005FF00000BDF800100A0402D5D3
:100F800087EA410101E006EA4101401CADF800108A
:100F90000828F1DB641EDDD26946084602F0A6F897
:100FA000BDF80000FCBD00000246002004E000BFC8
:100FB00012F8013B1844C0B2491EF9D27047000034
:100FC00070B5144A85B01088002413490194009428
:100FD000039420460494138807E00D8B009E35444B
:100FE0000095CD8B019E3544019515889D42F4D026
:100FF000401CC0B28028EED30098411107484180C0
:10100000848001984111064881830183818205B063
:1010100070BD0000F806002098020020C6050020E0
:10102000B404002030B50E4902880A800C4A438877
:10103000083A13800B1F808818802024151F2C80ED
:101040000020401C80B27328FBD341F211100880AD
:1010500044F64800108047F2480018802C8030BDCC
:10106000202C0140114944F648000880091D46F62D
:1010700048000880091D41F2111008800B48001F2C
:10108000018841F02001018009480021A0F8641086
:10109000A0F86210A0F86010A0F85E10A0F85C1034
:1010A000A0F85A100348418181827047182C0140F2
:1010B0009802002060000020F0B54D4B4D48002103
:1010C000DA7A0778802A27F001057CD31C684A4B1E
:1010D00002F01F0253F82220484B14421A6802D033
:1010E00042F0200201E022F02002454C1A60454EF9
:1010F00094F800C0444CBCF1020FB4F904403FD155
:10110000B3F808C0CCF3C00ECCF3002CE64537D0C2
:101110003A4D2C3D95F802C0BCF1000F04D0BCF153
:10112000010F0FD0A9702FE05FEA025C2CD55FEAB7
:10113000826C29D44FF0010C85F802C027F0040519
:10114000057021E05FEA025C1ED45FEA826C1BD569
:101150005FEA477C11D447F004070770B0F802C07B
:10116000BCF1000F03D0418027F0010704E0448068
:10117000002C02DD47F0010707700227AF7003E083
:1011800005704180318041811C4DC78895F84650DB
:101190000FB9002C15DC077BAF4212D1B0F90270F9
:1011A00007F26667BC420CDC184FBF895FEA477CD8
:1011B00007D45FEA877C04D45FEA427C01D5FF074D
:1011C0000BD0077800E00FE05FEAC77C05D027F07E
:1011D00001070770418031804181C4800573500947
:1011E00060F3CB221A60F0BD057041804181F0BDF3
:1011F000CC05002000090020FC8D0008980200208A
:10120000EF06002010010020C6050020080A00207B
:101210002DE9F04796B000240C940D940E940F9491
:1012200072B69048816941F400718161816941F42D
:10123000806181614FF4004002F01CFE8A4D002164
:101240002846FFF73FFB00212846FFF731FB874E7A
:1012500000213046FFF72CFB854F0021384600F077
:10126000BBF901204FF47041401C8842FCD3284652
:10127000FFF744FCB1463046FFF740FC384600F02B
:10128000B7F94FF46020CDE912048DF845400120F4
:101290004FF004088DF8440010948DF8508010A988
:1012A0002846FFF7BDFC01231A4605212846FFF713
:1012B00008FD0123022206212846FFF702FD012333
:1012C000032207212846FFF7FCFC012304220F21FB
:1012D0002846FFF7F6FC384600F08AF9684600F029
:1012E00032FA6148634E4C300090CDF80C80CDE965
:1012F00001648020CDE90440400006908000079002
:10130000202008904FF44050CDE909046946384642
:1013100000F0FCF901212846FFF7D4FA01213846F4
:1013200000F05AF901212846FFF7C2FA47F230517E
:1013300015941598401C15908842FAD3012128462F
:10134000FFF7FEFCADF82C40A04640F2DC5A4FF40B
:10135000007420E05046CDF854801599491C159131
:101360008142FAD330880D9908440D9070880E9907
:1013700008440E90B0880F9908440F90F0880C999B
:1013800008440C9001212846FFF7DAFCBDF82C0038
:10139000401CADF82C00BDF82C00A042DAD30D980B
:1013A000354A40F3CF1633480A3006830E9941F38D
:1013B000CF1444830F9941F3CF1383830C9941F3E6
:1013C000CF1CA0F804C0ACF5C05C40F2C371ACF512
:1013D0009B7C8C450ED2A6F5C856363E8E4209D26D
:1013E000A4F5C854363C8C4204D2A3F5C853363B0E
:1013F0008B4203D3D18841F48041D180D188490404
:1014000007D41E49028B21F85C2F428B4A80808BC7
:10141000888000212846FFF755FA0021384600F061
:10142000DBF800212846FFF743FA00214C464846E6
:10143000FFF73EFA0220C102401C8842FCD3284636
:10144000FFF75CFB2046FFF759FB384600F0D0F869
:10145000FFF742FA0A493C20087062B616B0BDE8B0
:10146000F0870000001002400024014000280140E5
:101470000800024012050020080A00205C0C002031
:10148000EC060020F0B5384B394C93F85650374BEA
:10149000042D5B6C1DD0256840F22D465D1B6560F8
:1014A00043F6FB25B3F5FA5F33DDB3F5FA4F30DCD5
:1014B00041F6AD17A3F5FA535F4306EBA7364FF499
:1014C000B5777B4305EBA31375105B10C4E9065396
:1014D00021E043F6D017102641F26205BB4218DB2B
:1014E00044F25067BB420EDAA3F5645345F24C67F1
:1014F000D03B5F4306EBA736A66140F624767343E4
:1015000005EB232303E042F24713A361194BE36188
:1015100001E0C4E90665A3695360E569401AD56036
:1015200010604543107C0541106A29181162D0698A
:10153000814200DD1062116A9069814201DB084638
:1015400000E01062206211684B43117A0B410841A0
:101550001918B2F91400884204DBB2F9120088426B
:1015600000DC08B2F0BD0000600000203C0100205B
:101570001401002085EB010010B54FF40054204603
:1015800000F0ACF8002813D00A49087840F00800B1
:101590000870204600F014F80021074800F01CF8FD
:1015A0000648C17E012903D10021C17601210177BE
:1015B00010BD00006606002044000240000B002021
:1015C000C10002D50249086070470249486070476F
:1015D00004040240000002400029016802D041F0EA
:1015E000010102E04FF6FE721140016070470000F9
:1015F00001684FF6FE7211400160002101604160F8
:101600008160C1603149314A0839904203D148684C
:1016100040F00F0006E02D4A1432904204D1486891
:1016200040F0F00048607047284A2832904203D1C9
:10163000486840F47060F5E7244A3C32904203D198
:10164000486840F47040EDE7204A5032904203D1A0
:10165000486840F47020E5E71C4A6432904203D1A8
:10166000486840F47000DDE7184A7832904203D1B0
:10167000486840F07060D5E7154A111F904203D1C9
:10168000086840F00F0006E0114A1432904204D17D
:10169000086840F0F000086070470D4A2832904218
:1016A00003D1086840F47060F5E7094A3C32904283
:1016B00003D1086840F47040EDE7054A503290428B
:1016C000EAD1086840F47020E5E700000800024015
:1016D00008040240406880B27047000001460020C4
:1016E000CA0001D5034A00E0034A12680A4200D04A
:1016F000012070470004024000000240002A0268F6
:1017000001D00A4300E08A430260704730B50368A5
:1017100047F6F07293430C6A8A682243D1E9044584
:101720002C4322438C692243CC6922434C6A2243D6
:101730008C6A22431A430260CA6842600A68826067
:101740004968C16030BD0021016041608160C160B5
:10175000016141618161C1610162416281627047E1
:1017600010B5114C8CB000212046FFF735FF204604
:10177000FFF73EFF0D4800900D480021CDE9010123
:101780006420CDE903018020CDE90501079108918E
:1017900009910A9169462046FFF7B8FF01212046CA
:1017A000FFF71AFF0CB010BD58000240043801408A
:1017B0008407002010B501218CB0084602F064FBBC
:1017C0001E4C00212046FFF707FF2046FFF710FFC1
:1017D0001B4800901B48019000211020CDE9020118
:1017E0008020CDE9041006910791089109910A9192
:1017F00069462046FFF78AFF012202212046FFF7B3
:101800007DFF01218DF82F1004208DF82D008DF81B
:101810002E100E208DF82C000BA802F019F80F20C6
:101820008DF82C000BA802F013F801212046FFF7D9
:10183000D3FEFFF795FF0CB010BD0000440002403E
:10184000043801402007002030B540F6AA21204A84
:10185000C184838B1488E31A9BB20F2B10D3128898
:101860008283037E002253B11A4BB3F90A30062B50
:1018700005DB194B1B78022B03D0002B00D182848F
:1018800030BD164B40F68B255B6CA3F22D14AC4299
:101890000FD2428B521C92B24283642AF0D364224C
:1018A0004283B0F924208A4201DA02EB21118184BB
:1018B00030BD41F29414A342FADBB0F92430002B7E
:1018C00002DDA3EB211100E000218184428330BDC1
:1018D000F806002060000020EF0600203C010020F8
:1018E00010B50446B0F9020043F69911484381133C
:1018F000E06840F26662504301EBA030E060B4F96A
:10190000001043F6991251438A13216940F266632D
:10191000594302EBA131216104F08CFC6061A18884
:1019200040F6AB2208444010A0F515415539E0625D
:10193000914205D9A0F5F851FF39521C91421DD2B0
:1019400049F25451884202DDA0F5204002E0A0F5A2
:10195000F850FF38206300EB400040F34F00208533
:10196000B4F924104A42904201DA104602E088425B
:1019700000DD0846E083228461848AE0A0F5FE420F
:10198000FF3A41F255518A4214D8A2F6AA202063A8
:1019900000EB400040F34F002085B4F92420514271
:1019A000E183884201DA084602E0904200DD1046F9
:1019B000404250E0A0F5D442AA3A8A4215D2A2F69B
:1019C000AA20206300EB400040F34F012185B4F9C9
:1019D00024004242E2832084914201DA104602E070
:1019E000814200DC0846608453E0A0F5AA42543AE4
:1019F00041F256539A4215D2A2F6AB20206300EB77
:101A0000400040F34F002085B4F924104A42904230
:101A100001DA104602E0884200DD08464042E083D9
:101A2000218419E0A0F5804241F254539A4215D224
:101A3000A2F6AA20206300EB400040F34F0121856D
:101A4000B4F92400E0834242914201DA104602E0F8
:101A5000814200DC0846208462841AE0A0F5285206
:101A6000AB3A8A4215D2A2F6AA20206300EB4000CE
:101A700040F34F012185B4F92400E08342422284DF
:101A8000914201DA104602E0814200DC0846404201
:101A9000A9E7B4F91E006FF4BF7148438013E080DA
:101AA000B4F92000484380132081B4F92200484350
:101AB0008013608110BD01210176704770470000DE
:101AC0001548164A4FF480410078042821D002F1CD
:101AD0003C03D08A9B88C01A00B22F2801DD001178
:101AE00008E0002801DD002007E00D4B984201DAF4
:101AF000184602E0402800DD40209389184400B2D7
:101B0000884203DC40F26661884200DA0846908130
:101B10007047918170470000EF060020B404002058
:101B2000C0FEFFFF38B54B484B4902880B889A1A14
:101B300092B20F2A71D30988484C01804FF0FF01FF
:101B4000E2884FF47A7355044FF4967002D516224A
:101B5000009103E0950403D515220091014670E041
:101B6000D50402D514220091F8E7150502D51322F9
:101B70000091F3E7550502D512220091EEE7950595
:101B800002D511220091E9E7D50502D51022009176
:101B9000E4E7150602D50F220091DFE7550602D5CE
:101BA0000E220091DAE7950602D50D220091D5E7C5
:101BB000D50602D50C220091D0E7150702D50B22DD
:101BC0000091CBE7550702D50A220091C6E7950799
:101BD00002D509220091C1E7D20702D00822009164
:101BE000BCE72289550702D507220091B6E7950781
:101BF00002D506220091B1E7D20702D0052200915A
:101C0000ACE7A27AD20702D004220091A6E7A2890B
:101C1000D40603D503220091A0E719E0140702D5EA
:101C2000022200919AE7540703D4940701D4D20703
:101C300002D00122009191E70020034602460146AE
:101C4000009002F0F5FDBDE838400248FFF72AB9E0
:101C500038BD0000FC090020F8060020080A00201A
:101C6000F0B55948594982880B889A1A92B29C2A31
:101C700064D30988818056490A880146002A0B7876
:101C800043F0020156D11646524A1C071568024617
:101C9000127822F0020274D54F4C0746E4887F7810
:101CA0005FEA845C02D547F0010701E027F00107F5
:101CB0004770A704477802D547F0020701E027F0F4
:101CC00002074770670401D4E70703D0477847F05D
:101CD00008074770640603D5447844F0040404E020
:101CE0001C0603D4447824F004044470EC0450D45B
:101CF000354C9A07247824F0100423D4324D4278CE
:101D00002F7A2D78012A45F0100514D0022A16D01A
:101D10002D4C042AA47804F1010C0CF0FF0C13D014
:101D2000072A25D0032A23D0052A21D0062A1FD02E
:101D300021F0100142E0B90702E00570F0BD39075B
:101D40000029FADB0470F0BDFA0601D41A060AD5A0
:101D50000170022C04D280F802C0BCF1020FF2D351
:101D600041F080012AE021F0100101708670F0BD81
:101D7000877A7F06F7D5032C04D8017080F802C05B
:101D8000F0BD0FE05107D8D51906D6D443F0800135
:101D900014E002704178CB0701D18907F0D522F019
:101DA00010010BE0E9040BD49907E9D4818AC82912
:101DB00002D2491C8182E3E743F00A010170DFE7A8
:101DC00002708682DCE70000D0060020F8060020C2
:101DD000FA06002098020020080A0020094944F66B
:101DE00048000880091D46F648000880091D41F694
:101DF000CC4008800348001F018841F02001018089
:101E000070470000182C0140084946F66800088019
:101E1000091D0880091D41F2555008800348001F24
:101E2000018841F02001018070470000182C01401A
:101E300010B5C28800210AB1032206E002890AB166
:101E4000022202E0428912B10122027000E0017018
:101E500004784FF4804344F6206244B1012C06D04C
:101E6000022C07D0032C01D14180818010BD43801A
:101E7000828010BD41F23331418040F6B731F4E742
:101E800030B5B1F86A5000231A240D22854202DCD5
:101E9000B1F9680030BD4D88854202DBB1F9000020
:101EA00030BD01EB82056D88854201DD144601E0FD
:101EB00013DA134604EB03024FEA52029A42F0D1BE
:101EC00001EB830231F8231054889288521A001BC8
:101ED000424301EB622000B230BD31F9220030BD37
:101EE000054920B1086940F0800008617047034847
:101EF000486003484860704700200240230167455E
:101F0000AB89EFCD06494FF47A70CA68D20705D085
:101F1000401E0004000CF8D1FF20704700207047DD
:101F20000020024012480321A0F14C0280F8361034
:101F3000002151810F4A11860F4A1186D162D18347
:101F40001184518481620D498A6CB2F5206F01DBE6
:101F5000A3228262897A11B1816A49428162C16A8F
:101F600041F39101816288030549086270470000CE
:101F700060000020980200201C0500203C01002089
:101F8000640800200449002048810881C8628862F2
:101F900002490862704700006000002088080020A5
:101FA000F0B53B4988894A89801A80B20F2866D3E8
:101FB00088894881CA8937480B3A272A26D28A78E5
:101FC00022BB8268364B42F480728260324A354CC2
:101FD000354D12785607314A0AD4344E3688168069
:101FE000334A12881A80334A12882280324A09E022
:101FF000324E36881680324A12881A80314A128848
:102000002280314A12882A8001228A702F4B304D5B
:1020100019469A7F0968802A32D302F01F0255F8C8
:10202000222011422CD0826822F48012184E826045
:10203000123614461215B778521C62F38617254AD9
:10204000B77093F816C01778BCF1800F27F002061E
:1020500008D30CF01F0C55F82CC011EA0C0F01D15D
:1020600047F0020616701A7E802A0DD302F01F0276
:1020700055F82220114207D144F400218160F0BDBF
:10208000826842F48012D1E724F40021F6E70000D0
:10209000EC060020980200203C010020AC04002047
:1020A000AE040020B0040020B20400209C040020F4
:1020B0009E040020A0040020A2040020A40400200C
:1020C000A6040020A8040020AA040020CC050020BB
:1020D000FC8D0008B404002070B520488189028975
:1020E000891A89B20F292FD3818901811C4B1D4880
:1020F00019465D7A06681C4C096846F00402802D7A
:1021000007D305F01F0554F82550294201D126F0C8
:10211000040202609A7B802A17D302F01F0254F84F
:102120002220114211D1026822F002020260DA7A02
:10213000802A0ED302F01F0254F82220114208D147
:10214000016821F00801016070BD026842F00202DE
:10215000ECE7016841F00801F5E70000EC0600201B
:10216000CC05002098020020FC8D0008F0B51D4C25
:102170001B4A4FF0010C94F83B5094F80AE01446C7
:1021800092F83C3094F838402B43651CEEB2154D64
:1021900095F83D700025BEF1FF0F0AD0BEF1000F8B
:1021A00006D18B4213D155700C2C01D282F83860C5
:1021B000F0BD834202D182F801C0F5E78B42F7D12E
:1021C0005570B80709E000BF82F83850F0BD83426F
:1021D000FCD1F84382F801C080070028F4D0F0BD9C
:1021E0003C0400203C010020F0B5CA78002502F034
:1021F0000F03D20601D58A7813430A784FF00F0EE9
:1022000012F0FF0F4FF001021CD004680F8802FA91
:1022100005F63740B74211D14FEA850C0EFA0CF79C
:1022200024EA070703FA0CF43C43CF78282F02D0A6
:10223000482F02D002E0466100E006616D1C082DC7
:10224000E4D304600C88FF2C1ED944685FF00006BC
:1022500006F1080702FA07F50F882F40AF420FD1A9
:102260004FEA860C0EFA0CF7BC4303FA0CF73C431A
:10227000CF78282F00D14561CF78482F00D1056154
:10228000761C082EE4D34460F0BD0000F0B5144C79
:10229000002801DAE36900E06368420D120185B2AB
:1022A000C0F301579540C0F30346032F05D0C20287
:1022B0000AD50322B240934307E023F070626368BB
:1022C00023F07063636002E0AB4343F0706201B1DE
:1022D0002A43002801DAE261F0BD6260F0BD00002F
:1022E000000001400246002092680A4200D001200E
:1022F000704741617047016170470AB101617047E1
:10230000416170470F4A104B92F838105B5C834272
:1023100001D1012004E00D4B5B5C834203D100201E
:1023200082F83A0070470A4B5B5C834201D18120FE
:10233000F6E7084B595C814201D18020F0E7032089
:10234000EEE700003C010020BC910008CE9100089F
:10235000C2910008D49100080A4810B501784FF0E6
:1023600000024C0708494FF0FF0389684FEA0171EA
:1023700005D5002901DA827210BD837210BD0029D3
:10238000FBDBF8E73C01002098020020F0B5194E75
:10239000194C0022E31CA6F1060CB75CA518ED78D9
:1023A000FF5C0D430F43BD421FD01CF80270FF5C61
:1023B0000F43BD4219D015460023A618F6780E43E8
:1023C000C6545B1C1CF80220DBB2062BF5D3C17887
:1023D00081700179C17000214218491C15711CF8E7
:1023E0000550C9B20629F7D3F0BD521CD2B2032A58
:1023F000D3D3F0BD8E8900083C04002010B50246FE
:102400000021064B06205C186478944200D10846EF
:10241000491CC9B20629F6D310BD00003C010020BA
:10242000214810B590F8671000222048012936D1C4
:102430001F49898899BB1F491E4B4C6C40F6B83127
:10244000B3F86E308C4227DD1B49097821BB90F828
:102450002711491CC9B280F82711C8291CD380F85C
:1024600027210146D0F82C4191F82811A34203DD21
:10247000052908D2491C01E041B1491E80F8281104
:10248000C9B2052902D3012180F82611191B074C76
:102490002C3C6162C0F82C31B3F5FA6F03D280F89E
:1024A000262180F8282110BD5C0C00209802002015
:1024B000C60500203C010020EF0600204FF4C0427A
:1024C0008260002141620E22828141F26202026139
:1024D000082282824FF46042C28201834FF0784228
:1024E000C0E9072140F6C41101807047B0F900101F
:1024F000B0F90220891A41600269037D4A431A41FA
:10250000436A13444362026A934200DD4262436AB3
:10251000C269934200DA42628268436A4A43017B9D
:102520000A410B41D118B0F918208A4201DA10464D
:102530007047B0F916008842FADC08B27047000014
:1025400010B514481449B0F88C200B889A1A92B22E
:10255000B2F5437F1DD90988A0F88C10B0F88A1015
:1025600020F8581F002242860C480D4CC2888280F9
:10257000C180C38983812489891AA4B2C4818160FE
:10258000E11A0161074A818AC182928A8282511AC4
:10259000816110BD3C010020F8060020240C0020C1
:1025A0001C0500206000002009480A49B0F8AA2054
:1025B0000B889A1A92B241F684639A4206D309882C
:1025C00020F8AA1F418881800021418070470000C7
:1025D0003C010020F80600200D480178C90702D010
:1025E0000C49098801E04FF6FA71C16509490120DB
:1025F0001039088007482438018841F00101018022
:1026000004481838018821F0180101807047000043
:102610003C010020240400400A49D1F8902012B166
:10262000521EC1F8902031F88A2F521C21F81A2925
:102630004A6A521C4A628A8F521C8A8701F8380CF7
:10264000704700003C0100201CB52D4890F83B303D
:1026500090F83C20934252D000248DF8044053401F
:102660008DF800309DF800300122012B08D09DF834
:102670000030022B09D09DF80030042B0AD00DE069
:102680001F498DF80420443108E01D498DF80420CD
:10269000463103E01A498DF8042048319DF80420A2
:1026A000012A2CD190F83D309DF80040154AA342F4
:1026B00017D090F83E309DF80040234208D0B0F883
:1026C0004C30A0F84A300B881488E31AA0F84C303C
:1026D00090F838302BB1B0F840301488E31AA0F8E5
:1026E000423012880A80A0F8402010F83E1F9DF862
:1026F0000020114300F801199DF8001001701CBD65
:102700003C040020F806002070B5344D40212846D6
:10271000FFF7E8FD840080212846FFF7E3FD44EA47
:102720004004A9152846FFF7DDFD0443E1B22C4C17
:1027300094F870508D4250D04D4084F87010012DA7
:1027400003D0022D01D0042D47D194F87400A84382
:1027500084F8740094F87320AA420FD084F8735060
:1027600094F8722001238B401A4207D11A4384F84F
:10277000722094F87110491C84F8711094F871104B
:10278000042928D330B1012811D002280FD0042801
:102790000DD012E01348C18821F04001C18020789B
:1027A000002184F83B1020F06000207005E02178C3
:1027B00041F02001217084F83B000B4994F83B0064
:1027C00091F82720904204D081F827000749202063
:1027D000087000F00DF884F84C5070BD00100140F6
:1027E0003C010020080A00205C0C0020EC060020C0
:1027F00070B50D4D40212846FFF774FD84008021FF
:102800002846FFF76FFD44EA4004A9152846FFF764
:1028100069FD04430548072100F8704F017100214C
:1028200041708170C17070BD001001403C010020FA
:1028300070B5344890F83A10CA43920761D001F05D
:10284000030280F8392090F83D305B061B0E80F8BB
:102850003D30012A01D0812A02D15B1C80F83D3035
:102860000278D2074DD0DBB203F00102C3F340047B
:10287000A24246D1B0F84E400025641CA0F84E405C
:10288000204CA0F8505090F83E60A47AB24202D09A
:1028900080F83E200DE0A607B6EB837F02D080F8DB
:1028A0003F5006E090F83F30642B02D25B1C80F86A
:1028B0003F3090F84030642B0CD25B1CDBB280F8C8
:1028C0004030022B06D204F00103934202D10222CF
:1028D00080F84020012901D0002912D190F8382039
:1028E000C16D00EB820291610163D0E906121144CF
:1028F000D0E908231A441144826A1144C26A11447F
:10290000416370BD3C010020FEE700002DE9F04F5F
:1029100000BF00209E4E9F4AA6F51271A6F5BE7913
:10292000A6F1440B06F1440E804601F5E074A1F1D6
:10293000780301F5457A1D5C15F0C00706D0402FDD
:1029400051D0C02F77D0802F76D004E115F01F052D
:1029500004D0154440F080072F7201E082F808800F
:10296000012826D0022824D0032822D0042820D0F1
:1029700008281ED010281CD0874D55F820C0DCF840
:10298000005054F820703D40CCF80050824D55F86E
:1029900020C0DCF8005056F820703D43CCF80050C1
:1029A0001D5CAD0659F820502F6813D53AF810C0B9
:1029B0003EE051F820502F6854F820C007EA0C0779
:1029C0002F6051F820502F6856F820C047EA0C07B6
:1029D0002F60E5E7DFF8B8C10CF1F00C5CF820C01F
:1029E00007EA0C077EE015F01F0504D0154440F0FF
:1029F00080072F7201E082F8088001281DD002288C
:102A00001BD0032819D0042817D0082815D0102867
:102A100013D0614D55F820502F6854F820C007EAB4
:102A20000C072F605C4D55F820502F685BF820C0D4
:102A300047EA0C0756E00BE056E051F820502F68AB
:102A400054F820C007EA0C072F6051F82050ECE73B
:102A500015F01F0505D0154440F0800785F821705A
:102A600001E082F82180012825D0022823D0032804
:102A700021D004281FD008281DD010281BD0464D77
:102A800055F820C0DCF8005054F820703D40CCF8D8
:102A90000050414D55F820C0DCF800505EF8207021
:102AA0003D43CCF800501D5CAD0615D53A4D3AF8C3
:102AB0001070CC3514E051F820502F6854F820C025
:102AC00007EA0C072F6051F820502F685EF820C0ED
:102AD00047EA0C072F60E6E72D4D3AF81070E03D0D
:102AE00055F820502F6036E015F01F0505D015442D
:102AF00040F0800785F8217001E082F821800128EC
:102B000030D002282ED003282CD004282AD0082820
:102B100028D0102826D0204D55F820C0DCF80050D1
:102B200054F820703D40CCF800501B4D55F820C0A3
:102B3000DCF80050164F883757F820703D43CCF82A
:102B400000501D5CAD06B1D4114F3AF81050E03F73
:102B500057F820703D60401CC0B21128FFF4EBAE66
:102B6000BDE8F08F51F820502F6854F820C007EAD4
:102B70000C072F6051F820502F68DFF814C00CF1BB
:102B8000880C5CF820C047EA0C072F60D9E70000EA
:102B900088900008CC050020848E00084FF407714F
:102BA000C1824FF45861018340F61451818370470C
:102BB000F0B5C48AB0F900608681B0F90250C581D1
:102BC000B0F904300227002101220382AB4204DB6A
:102BD000B54202DDC78042810CE0B34204DBAE4265
:102BE00002DDC78041811CE09D4205DBB34203DD6D
:102BF000C2804781018115E0B54204DB9E4202DDBF
:102C0000C280418105E0AE4205DB9D4203DDC1800B
:102C10004281078106E09E4204DBAB4202DDC180B7
:102C200047810281C388458900EB430700EB4505D6
:102C3000BB89AE899B1B0FFA83FEA0F812E00689C0
:102C4000AB8900EB460CBCF80CC0A3EB0C038382F1
:102C5000B0F91830B7F90CC0A3EB0C0CB4EB4C0F67
:102C600004DA80F82010A3F1A10113E0A64503DDEA
:102C700080F82010B9890BE026B1012E04D0022E75
:102C800010D004E0062100E0052180F82010A98979
:102C9000091B6D31418309B2B1F5586F04DB5B1E2E
:102CA000438304E00421F0E7002900DC4283418BE8
:102CB0008183F0BD0B49002288760A62CA614A62AC
:102CC000094A32F9103002EB40028B62B2F902205D
:102CD000CA62064A32F810000882A1F86000A1F822
:102CE00062007047EC010020E6910008DA910008CC
:102CF0002DE9F05FEF48F04982880B889A1A92B26A
:102D00000F2A44D309888180EC498246012708882C
:102D1000EB4CEC4E002578B3401E0880E573EA4981
:102D2000A5622068B1F90210430742F6AA2218D41E
:102D3000F38843F40053F380E34B1B789B0709D5DA
:102D4000A36823F08003A360A4F87C5084F87E502D
:102D500084F87F50C30404D484F8F070C4F8EC50B5
:102D600003E084F8F050430707D4914205DB84F870
:102D7000F470A4F8F25004E010E084F8F450430733
:102D800003D4914201DBC00703D084F81151BDE8A0
:102D9000F09F84F81171A4F81251F8E7B4F8180103
:102DA00043F69821884202D2401CA4F8180101F091
:102DB00055FDDFF81883DFF8FCB298F85000ABF14E
:102DC000180B10B1FEF778F905E09BF8001021F020
:102DD00001018BF8001098F8630010B1FEF732F88B
:102DE00008E0A068C10502D520F0080001E040F02D
:102DF0000800A060FFF714FB00F0A4F9B44841F20A
:102E00006801436C4FF400608B4201DBB14904E080
:102E1000B3F57A6F02DAAF49091D086098F85100DE
:102E2000C646C107DFF89882AB48DFF8B092A8F138
:102E30002C0839D0817B802932D3217889072FD47F
:102E4000E27B88F80520A04A414692F800C02CF0A9
:102E5000020C82F800C0ABF80250CBF814509BF87B
:102E600000C02CF0010C8BF800C0B279520612D4CD
:102E70004A8941F2883C624503D2521CA8F80A20D4
:102E800012E040F63C70834201DD0020DEE00420C9
:102E900088F80370DAE0CD700020A8F80A50D5E079
:102EA00088F80350A8F80A50A1680A0501D508203F
:102EB000CCE09EF83FE05FEACE7240D0E27B88F83B
:102EC0000520437A802B59D323785B0730D4F388CD
:102ED0009B0403D521F02000A06030E0ABF8025045
:102EE000CBF814509BF800C041F020012CF0010CED
:102EF0008BF800C0A160C17D802909D301F07F0358
:102F000000684FF00041D940084201D1277100E02C
:102F100025712079C00702D15FEA8E7005D50320A4
:102F2000032A01D088F8087090E00020A5628DE0A7
:102F300021F02000A060F08820F40050F08094F888
:102F4000260101281FD094F8462043F233304FF475
:102F50008047D2B143F69911012A2CD099F800206C
:102F60005F48C2F38102012A28D0022A26D090F8B5
:102F70005600A4F81471042831D025E0206840F0F0
:102F800004002060A6E7092060E099F80010C1F372
:102F90008101012909D002290AD042F6B86100BF97
:102FA000A4F81411A4F8440010E042F6CC41F7E76D
:102FB00042F26661F4E7A4F8140110E0A4F8147179
:102FC00090F8560004280AD0A4F84470FEF774F86C
:102FD0009BF80010C90705D0BBF8021004E0A4F864
:102FE0004410F3E738488188AAF8121008B2B4F9FF
:102FF00044104843C0F38F314046A8F81210B9423C
:1030000000D9478237490978C90605D5428A41F275
:1030100033318A4200D241822189C1F3C002C1F317
:1030200000218A4205D1428A40F6CC418A4200D929
:103030004182B17AC90700D04582B8F81200A06277
:1030400000287FF722AF2848057002209AF81A104E
:1030500099B9022824D080B11D490B789D0608D566
:10306000B5796D0605D51F4D2D78ED0965F38613ED
:103070000B70F18821F40A61F1801549496C4E29E1
:103080000ADBF1880B0607D521F08001F1800E499B
:103090000B7823F002030B708AF81A00E07376E6CF
:1030A000B9F83830002BD7D143F69823A9F8383037
:1030B000D2E7000018090020F8060020FA060020D8
:1030C00098020020080A0020C60500205C0C0020A1
:1030D0003C010020100C0140CC050020B40400206D
:1030E00060000020D00600200C07002070B50023EF
:1030F0000C8863F30F02012505FA03F6344206D06B
:10310000C3F10F0605FA06F1114361F30F025B1CD0
:10311000102BF1DB028070BD70B500230C7863F3D7
:103120000702012505FA03F6344206D0C3F107066B
:1031300005FA06F1114361F307025B1C082BF1DB72
:10314000027070BDF0B51F4890F866301E48012B24
:10315000816821F4006232D11C4BDE8874062ED4C3
:103160001B4D0F054FF00004B5F902501ED4194A4B
:10317000526C642A11DC40F6386295420DDAB204D2
:103180000BD4027852070ED4B0F8D42040F6B835EC
:10319000AA4203D2521CA0F8D420F0BD41F4006131
:1031A00081605C81F0BDA0F8D440F0BD41F2CD015A
:1031B0008D42FADD997AC907F7D18260F3E7826020
:1031C000F0BD00005C0C002098020020080A0020DE
:1031D000C60500203C010020F0B5364D364F0446B0
:1031E00095F83B0097F83B1023780843EE1C627873
:1031F000834205D1E0781146FEF7B8FF207908E058
:1032000094F802C084450CD1E1781046FEF7AEFF79
:10321000E07905F82F0F2878805D6870287BE877C3
:10322000F0BD82421DD161461846FEF79FFF95F81A
:103230004E1095F83B00814207D1B97A09B1A179C6
:1032400000E0617985F82F101EE06978012901D02E
:10325000A17922E0617927E0297841F00401297001
:1032600012E0E1788142DBD119466046FEF77EFF2D
:1032700095F84E1095F83B0081420AD1B97A09B110
:10328000617ADFE7217ADDE715F82F1F895D697024
:10329000C5E76978012906D0617A85F82F10B97AD7
:1032A0000029F1D1D8E7217A85F82F10B97A0029C1
:1032B000EAD0D1E73C0400203C0100200B48017813
:1032C00021F0020100F8381B002100F8181941779D
:1032D000817733218185418508214184012100F8CE
:1032E0001F1C034880F83910704700003C04002080
:1032F0003C0100200D4900B50B4851F8012F40F862
:10330000032F89888180084801210930FFF73EF8A2
:10331000054802211330FFF739F8034804211D3016
:103320005DF804EBFFF732B83C0400203C010020BC
:10333000094944F648000880091D46F648000880FF
:10334000091D41F2111008800348001F018841F057
:103350002001018070470000182C01402DE9F04742
:10336000664C674B0025A0780126654A1033052876
:103370007ED2DFE800F00313113E1100108820F028
:10338000010010801D805F480580001F0580001F20
:103390000580FFF7CDFFA670BDE8F087594941F2DF
:1033A00044401C390880574945F6580024390880A4
:1033B000091D47F25800088052492020283908800A
:1033C0000020401CC0B27328FBD3FFF7B1FF4C496B
:1033D00084F85C502C3147F69060088048481430DF
:1033E00006801D80108840F0010010800220A0702F
:1033F000D2E700215FF0010004EB410204EB40033F
:10340000B2F85020B3F850309A4200D20146401C26
:10341000C0B20628F0D33C48405C84F83900FFF77E
:103420004DFF1D2000F0F3F900F076F8374E3848D4
:103430004FF4807996F83B10012904D002291BD063
:10344000042930D047E040218046FEF74BFF87003B
:1034500080214046FEF746FF47EA4007494640467E
:10346000FEF740FF074347F0010084F83B0000E00F
:103470003DE0224809302CE040218046FEF732FF33
:10348000870080214046FEF72DFF47EA4007494666
:103490004046FEF727FF074347F0020084F83B0051
:1034A0001648133015E040218046FEF71BFF8700C9
:1034B00080214046FEF716FF47EA4007494640464E
:1034C000FEF710FF074347F0040084F83B000B4869
:1034D0001D3002F099FD94F82F0086F838001D2069
:1034E00000F0ABF90420A0700A48057054E710887A
:1034F00020F0010010801D80A5704DE73C040020E5
:10350000000800403C2C0140948900083C01002048
:1035100000100140EF0600202DE9F041344C14F872
:103520002F0F344DE07240212846FEF7DBFE860067
:1035300080212846FEF7D6FE46EA4006AF153946FA
:103540002846FEF7CFFE0643207BF1B22F3C814296
:1035500015D084F83C0040212846FEF7C3FE8600C3
:1035600080212846FEF7BEFE46EA40063946284638
:10357000FEF7B8FE064384F83B60FFF765F81E4D82
:1035800095F83B00012827D0022828D0042829D00C
:10359000174894F83B102730085C04F8300F14F8F3
:1035A0000109FEF72BFF04F82F09A87A00B10120CA
:1035B000607001F0DFF994F84E0094F83B108842F7
:1035C00006D094F83800062802D2401C84F838004F
:1035D00084F84E10BDE8F0810548093004E0044845
:1035E000133001E002481D30BDE8F041FFF7F4BDA3
:1035F0003C040020001001403C0100202DE9F04176
:10360000524991F87200AA287ED191F8730055288A
:103610007AD14F4C00200A5C2254401CC0B274285E
:10362000F9D34C4E2069C6F80100A08AA6F805001F
:10363000D4F81600F060D4F81A003061D4F81E00F7
:103640001234706102F086FC4349608A888102F07E
:103650009BFC207D123CC007307802D040F0040073
:1036600001E020F004003D4930704FF480403C4DB3
:10367000886114F8280F85F82000608B6880A08B83
:10368000A880E08BE880208C2881608C354F688191
:1036900094F8240087F8D20014F8011C304686F80C
:1036A0003B100026C0F89460FFF724FE2E48A18E40
:1036B0000183E18E4183218F818394F84210283C5D
:1036C000012908D0022901D0032909D0297821F045
:1036D0000C01083107E0297821F00C01091D02E0F6
:1036E000297841F00C01297094F86E20012162B113
:1036F000012A01D0022A0BD087F8461094F86430D2
:103700001A4A4BB1518108E014E087F84660F5E7AA
:10371000022287F84620F1E7568194F870100129BB
:103720000AD094F86D1051B101290BD04FF480519B
:10373000A0F87610BDE8F08144F21C71F8E74FF470
:103740000051F5E741F25551F2E7000000FC000896
:103750005C0C00203C01002060000020F40B0020E5
:10376000B4040020980200201C050020080A002054
:103770007CB50121082000F0ABFB4FF48070ADF860
:10378000040010248DF8074001208DF8060001A9DF
:103790001548FEF729FD0121092000F099FB0121C0
:1037A0001248FEF773FD0820ADF8000004208DF8E4
:1037B00003000F4E03258DF8025069463046FEF790
:1037C00013FD08213046FEF794FDADF800408DF85A
:1037D00003408DF8025069463046FEF705FD102182
:1037E0003046FEF786FD7CBD00140140000230002B
:1037F000000C0140FEE7704700F01F0201219140DC
:103800004009800000F1E020C0F88011704700F00E
:103810001F02012191404009800000F1E020C0F822
:103820008011704700F01F02012191404009800083
:1038300000F1E020C0F80011704700F01F020121E4
:1038400091404009800000F1E020C0F8001170476D
:1038500070B50F23C47801780122F4B1144C2468A8
:10386000457804F4E064C4F5E064240AC4F1040675
:10387000E3408478B5401C402C4301F1E021230152
:1038800081F80034007800F01F018A404009800070
:1038900000F1E020C0F8002170BD01F01F0082405F
:1038A0004809800000F1E020C0F8802170BD0000D0
:1038B0000CED00E00249084302490860704700002F
:1038C0000000FA050CED00E02DE9F05F00261D2058
:1038D000FFF792FF6C4CDFF8B4B1A4F1B000A77E03
:1038E00090F83810DFF8A8E1DFF8A8A100258F4292
:1038F0007ED0E776A176626A036B5A434FEA12499B
:103900009BF80820120702D51EF8012000E00A46A5
:1039100094F812C0BCF1010F09D004EB4206B6F9CD
:1039200002C0C4F828C0B6F90460E6620CE043F6B1
:10393000FF7CC4E90A5C90F83DC05FEACC7C01D012
:1039400012B102E0052A00D1012600EB47074FF033
:10395000804CBF893F04B7FBF3F3E361476BBCFBCB
:10396000F7F7276294F813C0BCF1000F06D0BCF142
:10397000010F05D03B4403EBD3735B10636201E09E
:103980003B466762DFF810C14FF6FF7707EA83070F
:10399000ACF808709AF8007090F80A8090F83DC072
:1039A000082F08F003070CF0030C05D067450BD176
:1039B000B8F1000F05D008E0674505D0B8F1000F59
:1039C00003D05B42636200E06562C6B1636A002BAC
:1039D00003D006DD228D05E00AE0304B33F81220DB
:1039E00000E0A28DA4F86020227822F0200222704C
:1039F0009AF80020042A07D0082A05D012E0B4F86B
:103A0000603003EB0902EDE780F8405065629BF8F7
:103A10000800000701D51EF80110204830F81100F9
:103A2000A4F860001E49606A09883E314843B4F832
:103A3000601001EB204006B21D20FFF7F3FE606A24
:103A4000002807D021784FEA81600ADD002804DAD7
:103A5000A08D09E0B4F8600006E0E06AB04208DB3F
:103A60000CE0002802DA208D208208E0A06AB04233
:103A700004DD208241F02000207000E026822575C0
:103A800065752586BDE8F09FEC01002098020020B6
:103A9000C8910008EF060020E0090020DA91000834
:103AA0002404004043184FF48042934210DD9042BA
:103AB00002DD104600210BE0914202DD002011469C
:103AC00006E08003B0FBF3F000B2C0F5804109B21C
:103AD00041EA0040704700002DE9F043002340F226
:103AE000AE440E2544600362058144F24C2608274B
:103AF000C6600782DFF8349043F6FF7CA0F812908E
:103B0000A0F814C04FF070484FEA8C32C0E906822A
:103B10004C600B620D81CE600F82A1F81290A1F86B
:103B200014C0C1E90682BDE8F083000000C0FFFFB9
:103B300000214162094981600E2181814FF6BF5108
:103B40000161082181824FF44041C18243F6FF7137
:103B500001830907C161024901627047638A01005C
:103B600000C0FF0F064941F6A260088005480168C1
:103B7000054A01F4E06111430160BFF34F8FFEE796
:103B8000442C01400CED00E00400FA0538B5012199
:103B90000D2000F09DF94FF4E060ADF8000018240E
:103BA0008DF8034003258DF8025069460D48FEF755
:103BB0001BFB4FF46040ADF800008DF803400A4C49
:103BC0008DF8025069462046FEF70EFBA014ADF8B2
:103BD000000048208DF8030069462046FEF704FBEC
:103BE00038BD000000080140000C0140F0B5012183
:103BF000CE028DB0304600F06BF9594F384601F0D7
:103C00002BFB08A801F054FD4FF45860ADF82400D8
:103C10000024ADF820402020ADF82200ADF8264069
:103C200008A9384601F0F6FC0021384601F049FDAC
:103C30004FF6FF71384601F04EFD01220021384653
:103C400001F0DAFC0121384601F0C2FA04A801F0C3
:103C5000DAFAADF810607010ADF81200ADF814404B
:103C6000A220ADF816007000ADF81800ADF81A40AB
:103C7000ADF81C4004A9384601F0B4FA6025ADF84F
:103C80000050ADF80440ADF80840ADF80C40ADF878
:103C90000240ADF80640ADF80A40ADF80E40694666
:103CA000384601F099FB6946384601F0DBFB69466E
:103CB000384601F021FCADF800500125ADF8045064
:103CC00040F61450ADF80600ADF80840ADF80C40D1
:103CD000ADF80250ADF80A40ADF80E4069463846DE
:103CE00001F04EFC0121384601F096FA08213846D1
:103CF00001F0B2FB3146384601F0F4FB08213846AA
:103D000001F038FC3146384601F06CFC7021384631
:103D100001F075FC18208DF82C008DF82D408DF8E1
:103D20002E408DF82F500BA8FFF792FD0C480C3059
:103D3000018841F08001018009481430018841F078
:103D400001010180001F04800121384601F06EFA54
:103D50008DF828500121384601F072FA0DB0F0BDFF
:103D6000002C01407047000070B50189C1EB411182
:103D700001EB4101CA0B42810B49104603F0C6FC1E
:103D800009480C38B0F90C200168B0F90E4001FB6D
:103D900002F54368614303FB145503FB0211AD13A5
:103DA0008913C0E9055170BDEC09002040F21341B0
:103DB0004160082181608621C1604FF4804101612A
:103DC0004942416100210162C1627047016270474E
:103DD00010B501884288891A09B20183B1F5005FE4
:103DE00002DBA1F5804104E011F5005F02DC01F582
:103DF00080410183B0F9182041685143C161836853
:103E0000846A5343C2681B12624303EB2222036A93
:103E10001A44114402628A13426241698A4203DBF6
:103E200001698A4200DC11468A1AC0E90A21028E21
:103E30004FF40373594302EBA13202860B4A127806
:103E4000082A04D10A4AD36E03EBA131D166B0F936
:103E50003010B1F5804F02DDA1F5804103E000296B
:103E600002DA01F58041018610BD0000EF06002056
:103E70001C0A0020034A516821F44041014351606B
:103E80007047000000100240044A0029516901D027
:103E9000014300E08143516170470000001002407F
:103EA000044A0029D16901D0014300E08143D16176
:103EB0007047000000100240044A0029116901D037
:103EC000014300E08143116170470000001002408F
:103ED000044A0029916901D0014300E081439161C6
:103EE0007047000000100240044A0029D16801D048
:103EF000014300E08143D1607047000000100240A0
:103F000030B524494A6812F00C03234A03D0042B2D
:103F100001D0082B26D002604A680F231F4C03EA09
:103F20001212A35C0268DA4042604B68072505EA7A
:103F30001323E35C22FA03F383604B6805EAD3237F
:103F4000E35CDA40C2604B68032403F4404104EAB6
:103F5000933303EB9161114B1B1F595CB2FBF1F1E1
:103F6000016130BD4A680E4B1A404B68140103F4DE
:103F7000803303D5C2F38342113202E0022404EB02
:103F8000924213B14B689B0301D5064B00E0024BF4
:103F90005A43C0E70010024000127A0004000020DB
:103FA00000003C0800093D002DE9F041274CA61512
:103FB00040212046FEF796F9850080212046FEF735
:103FC00091F945EA400531462046FEF78BF9054355
:103FD000EDB240212046FEF785F98700802120467A
:103FE000FEF780F947EA400731462046FEF77AF9A6
:103FF0000743F8B2A842DBD140212046FEF772F910
:10400000870080212046FEF76DF947EA40073146D8
:104010002046FEF767F90743F8B2A842C8D140210D
:104020002046FEF75FF9870080212046FEF75AF907
:1040300047EA400731462046FEF754F90743F8B2F5
:10404000A842B5D12846BDE8F0810000001001402B
:1040500010B50268416802FB02F301FB01330D4C0D
:10406000A34211D91B0E0D3B0B4C9BB212B234F87C
:10407000133009B25A43594342F38F3241F38F311F
:10408000C0E90221012102E0C0E9022100210174FE
:1040900010BD0000C1B98A0DE48600082DE9F05F6B
:1040A000FD48FE4902880B889A1A92B20F2A76D3ED
:1040B00009880180FA4802468189D2884B0703D4D7
:1040C0008B0701D4CB0702D042F4007201E022F446
:1040D0000072C2808346080702D45846C90604D538
:1040E000BBF8061041F0010102E0C18821F0010196
:1040F000ABF80610EA48FDF79BFEEA484FF480490A
:10410000B0F93A10494502DA491C418701E0A0F8AC
:104110003A90E54E41F6CC41E44CB06C884203DD68
:10412000A06820F01000A060E14AE24FE248118848
:10413000002511B1491E118008E0E18F41B1491EEF
:10414000E187DE490A7822F002020A70E5732DE069
:10415000BBF806104B0419D4BBF80C20D30615D4B9
:10416000120713D40A0611D48A060FD40A050DD4F7
:104170004A0603D5D24A1278120607D54A0705D453
:10418000CA0503D40A0701D4C90609D5CD49E57388
:10419000CD4A3D70CD83158081F82A5007E07BE041
:1041A0003978012903D10178062900D13D70397889
:1041B000DFF8F8A2C54BAAF12C0A4FF001080A2932
:1041C00078D2DFE801F0F3690569F2F16977D5EC9F
:1041D000E07B09281AD0DFF8F8B202286CD0B4F8D6
:1041E000400010B39BF8680040F63A22012822D024
:1041F000C4F8D85084F8EA50CAF82050B4F9301006
:1042000001F21D50904226D8102325E0A2484430E8
:10421000FEF754F9FDF786FE716CCAF8281041F2DA
:104220007C510920CAF8181084E1AA48018B218624
:10423000A4F8408015E0A848C4F8D80084F8EA80C3
:10424000B4F9301001F21D53934201D8102300E05D
:104250002023102202E020231022002000F0F4FA94
:1042600020869BF868309D49012B736C40F2DC502E
:104270004FF4927212D0834204DA9648B0F90A00E1
:10428000904212DBB4F8402040F6C410521C92B2A7
:10429000A4F84020824208D2BDE8F09F8342FBDAB6
:1042A0008C48B0F90A009042F6DA3D7084F8EA5082
:1042B0004D83F1E7B8E0FFE7706CCAF828008AF890
:1042C0000780874FA4F8405084F8EA50797F56461B
:1042D00099B1F87FD8B3208DB4F9301000B20A2319
:1042E000052200F0B1FA2086FD777D77B4F9300021
:1042F000484539DDA4F83090CEE700B2794901F0A5
:10430000EFFBA4F8E400A16A814200DA084600B29B
:10431000B0829BF84D100029B4F9301002D036233A
:10432000052201E0A323102200F08EFA2086B4F9C2
:104330001601B4F9141188420ADA317901F1010148
:10434000C9B231710429D1D33571401C02E007E0B4
:1043500003DD801EA4F81601C8E7A4F81611C5E70E
:1043600040F266602086C1E7002895DA258693E74B
:104370005D49D4F8DC00884202D2401CC4F8DC005D
:10438000E07B082803D1D4F8DC00884203D33D70D9
:10439000C4F8DC5080E7BDE8F05F02F0F9BBE07BD9
:1043A000092804D0258623E122E01DE024E0DAF884
:1043B0001C005746401CCAF81C00022809DD388D35
:1043C000012301B2388B052200B200F03DFAFD61F5
:1043D000B8623148398D44300180B6F844104180CC
:1043E000FEF784F8208657E7BDE8F05F04F03CB89C
:1043F000187809284FD04FE73C490A78521CD2B2AE
:104400000A70C82A10D33A4A92F800C0BCF1010FD2
:104410000AD115700D70BBF80620364922F40062EF
:10442000ABF8062081F80080E17B891E082967D25D
:10443000DFE801F006A6E0F205FC8204E6E62BE7E1
:10444000FDF78AFF3078400611D52B488078042884
:104450000DD0706C82280ADAB07A96F83D1000F020
:10446000030001F00301884201D001F039FD3878E2
:1044700006288FD086F83F50B06C164940F31100E3
:10448000C86281031D480162FDF74CFD8AF8078070
:10449000B4F8140135E0ABE018090020F80600205C
:1044A000080A00201C0500203C0100209802002082
:1044B000FC060020EF060020F0060020C6050020C4
:1044C000D0060020AC0800201E000020540200206E
:1044D0005C0C0020600000209AF9FFFF8809002092
:1044E000240C0020D8880008C0D40100150000204A
:1044F00016000020140000203C0400208808002042
:1045000094E0A4F81601706CA4F88250B0F5437FD3
:10451000A4F880905FDCA16821F48061A16040F282
:104520008A21884204DA3078400601D402F01CFA6D
:10453000A06858E03870AFE6716CB1F5437F04DADB
:104540000178062901D0057069E03C48017821F026
:1045500040010170FDF7E6FCA4F81691FDF7FCFEA2
:10456000374810F8281F21F0010101703549C4F8BF
:10457000DC500D6234490D620821397045648BE6C8
:104580009BF80600C006D6D4706CB0F57A7F2FDD9C
:10459000FDF7E2FE3078400611D52C4880780428DB
:1045A0000DD0706C82280ADAB07A96F83D1000F0CF
:1045B000030001F00301884201D001F091FC86F86C
:1045C0003F50B6F84800208601B2494501DDA4F805
:1045D0003090FDF7A7FCA06840F48060A06096F8DA
:1045E00038100529A7D140F01000A0600220A1E7F3
:1045F0003D7051E6716CB1F5437F02DA017806290E
:10460000A1D1BBF8061021F02001ABF80610FDF790
:10461000A3FE04208EE7FFE70078062802D087F883
:10462000008039E609201870052083E707498D705E
:104630000570074880F8565098E60000FE060020F6
:104640001C0A002064080020880800203C04002088
:104650006000002030B585B001210420FFF738FC50
:104660004FF40040ADF8100048208DF8130004A965
:104670001848FDF7B9FD01210846FFF711FC40F687
:104680008C20ADF8040003240020ADF80040ADF804
:104690000200ADF806004FF080456946284600F05C
:1046A000B9FF1C208DF80C008DF80D408DF80E40E0
:1046B00001208DF80F0003A8FFF7CAF80122114668
:1046C000284600F081FE0121284600F0AFFD05B02C
:1046D00030BD000000080140704700002DE9F041A6
:1046E000304CE07800285AD12078002857D0401E5E
:1046F00010F0FF00207052D14FF49670208272B6F5
:10470000294F45F2AA50A7F872000020FDF7E8FBF8
:10471000264D13202860FDF7F5FBA8BB3420E86088
:1047200002202861224E6E61286940F04000286115
:10473000FDF7E8FB40BB00211E4A08465FEA25530F
:1047400012F800C0BCF1FF0F00D00121401C80B264
:104750009842F5D3C1B9C4E9067639260127A06984
:1047600010F8011B10F8012BA061E06901EB022198
:1047700002886A612F6120F8021BE061FDF7C2FB2D
:1047800010B9761EB6B2EAD20120FDF7A9FB62B6D7
:1047900001F0FAFB0848816821F480418160BDE89E
:1047A000F0810000EC0600205C0C0020002002409C
:1047B00000FC000800FC000898020020194801686D
:1047C00041F010010160016821F0030101600168FE
:1047D00041F0020101601448416841604168416054
:1047E000416841F480614160416821F47C1141607D
:1047F00041680E4A11434160016841F080710160D7
:1048000001688901FCD5416821F0030141604168DC
:1048100041F0020141604168C1F381010229FAD1EE
:1048200070470000002002400010024000002808ED
:1048300030B5044C039D6080A180E28023816581B6
:1048400030BD0000FC0900200A44824201DA10B2A7
:104850007047C91A8142FBDD08B27047F0B53E4887
:10486000DFF8F8E03E4CC17F467A056800233D4AF8
:104870003D484FF0010C802925D301F01F015EF85F
:1048800021100D420146096802D041F4805101E037
:1048900021F480510160CF0411D48F040FD5977A91
:1048A000FF0705D05381277827F00207277006E01D
:1048B00090F846709FB1012F14D080F846300F0B4E
:1048C00067F34D310160802E25D306F01F015EF89D
:1048D00021100D42016809D041F0040108E080F880
:1048E00046C0ECE7022780F84670E8E721F00401B3
:1048F00001604D070BD44D0509D5957AED0706D01B
:104900005381257825F002052570C0F898308C0871
:1049100064F38A210160917AC90718D1134991F88B
:104920006410012913D11249496C32290DDC017838
:1049300049070AD50189090507D4D0F8981047F22C
:104940003054A14204D9A2F80AC0C0F89830F0BD92
:10495000491CC0F89810F0BDCC050020FC8D000863
:10496000C6050020080A0020980200205C0C0020E8
:104970003C01002010B5FCF7FBF90F48018821F03D
:10498000020101800C49183109880C4A928E1144A9
:10499000094A3432118008490C390A8842F0010270
:1049A0000A80011D0A884FF6ED531A400A800188DB
:1049B00041F01201018010BD0C0400403C040020B5
:1049C00006480188491C89B20180B1F57A7F04D379
:1049D0004188491C41800021018070471007002058
:1049E0000F4810B5016841F00101016041680D4AAE
:1049F0001140416001680C4A11400160016821F4D6
:104A000080210160416821F4FE0141604FF41F01E3
:104A10008160FFF7D3FE05494FF00060086010BDCC
:104A2000001002400000FFF8FFFFF6FE08ED00E076
:104A30002DE9F0412F4D28884FF00004000629D5BC
:104A4000FCF710FB2C4A2D4807231778C8262C4961
:104A5000012F22D02B4FB7F806C0BCF1000F3ED07B
:104A6000B0F80CC04CF0080CA0F80CC0B0F806C0B0
:104A70002CF4006CA0F806C0886820F00400886060
:104A8000FC801370CE8700204FF49661401C80B2EA
:104A90008842FBD32C80BDE8F0811B4F97F800C003
:104AA000BCF1010F0FD0BCF1020F11D0B0F806C05D
:104AB0004CF4006CA0F806C0886840F004008860E0
:104AC00005203870DDE7B0F80CC04CF0080C03E0AE
:104AD000B0F80CC04CF0100CA0F80CC0F0E70B4F75
:104AE0003C70C78847F40067C780886840F00400BE
:104AF0008860C6E7102C0140EF060020080A00205D
:104B00009802002018090020F00600200D07002060
:104B1000704700002DE9F0434FF08040018A21F0FA
:104B200001010182AC48007800287CD1AB4FF87BB2
:104B3000002878D1AA48406C322874DCA9488068E3
:104B4000DFF8A4924104A94DB9F804004FF0000425
:104B500003D4401CA9F8040028E1002874D0297867
:104B6000012611B1012912D017E14946B0F5BE7FE7
:104B7000FAD92E70CC718C71EC702C72287A0A18CC
:104B8000401CC0B2147228720F28F7D305E1B9F89F
:104B900002204946824201D9EE7100E0EC71924850
:104BA0008A7908300F2A15D2CB79082B0BD2C3F1A2
:104BB0000708EB7912F800C003FA08F363441354B2
:104BC000CA79521CCA71CA79082A03D18A79521C3F
:104BD0008A71CC7199F80610C8460F2973D10D213E
:104BE000FCF7AAF9A881010A6970C0B2A87088F818
:104BF000064098F816208A4265D198F8151081422F
:104C000061D198F80BC07A49032302227948BCF19C
:104C1000000F10D0BCF1010F02D0BCF1020F14D074
:104C200080F86A2000E0CBE091F800C02CF00C0C7A
:104C30000CF1080C0FE080F86A6091F800C02CF0CD
:104C40000C0C0CF1040C06E0A9E080F86A3091F835
:104C500000C04CF00C0C81F800C098F80C10B6EBBA
:104C6000111F04D180F86E4087F846400EE0B2EB89
:104C7000111F04D180F86E6087F8466006E0B3EB40
:104C8000111F03D180F86E2087F846200B0717D03C
:104C900001F00F01012901D0022915D080F86C60C4
:104CA0002C7198F80D102A7906FA02F30B406B71FB
:104CB000082A44D2DFE802F00B124319242F363DB4
:104CC00080F86C40ECE768E080F86C20E8E713B10E
:104CD00080F8704033E080F8706030E013B180F805
:104CE00050602CE080F8504029E023B180F86560E6
:104CF00087F8036123E080F8654087F803411EE0F0
:104D000023B187F8F54080F84D4018E087F8F5604A
:104D100080F84D6013E013B180F868600FE080F810
:104D200068400CE013B180F8666008E080F86640E7
:104D300005E013B180F8676001E080F86740521C1D
:104D4000D2B22A71082AAED398F80E102A4A8B07DD
:104D500005D587F8F16080F86460568104E087F833
:104D6000F14080F864405481C90702D080F829409E
:104D700001E080F8296098F8111000F86D1FC278E2
:104D80001E48012A1ED001B3012921D04FF48051C1
:104D9000A0F876101A493C200870A9F80240A9F83A
:104DA0000440B9F80210491CA9F80210B9F8021021
:104DB000B1F5FA7F04D940F2F511A9F802102C7070
:104DC000BDE8F08344F21C71E2E74FF40051DFE7E5
:104DD00041F25551DCE70000EF0600209802002068
:104DE0003C01002000100140440C002088060020F7
:104DF000B40400205C0C0020080A00201C050020E0
:104E0000EC0600202DE9F05FFDF7A6FA8E4D28880C
:104E1000A5F10406C0070AD0308820F008003080D1
:104E2000288820F00900288001F09EFDD9E028881C
:104E3000DFF81892DFF81882864C80071AD5B9F887
:104E4000001041F00101A9F80010B8F800008049F5
:104E500014315030088028884FF6F95108402880D6
:104E6000308840F004003080FFF79EF884F83C0062
:104E7000BDE8F09F2888784F4007288871D520F03A
:104E800004002880FFF790F894F83C108142EFD19D
:104E9000308820F004003080FDF736FC2078410691
:104EA00005D594F84C1094F83B209142E0D0397825
:104EB000400621F00201397004D5FEF72DFB97F86A
:104EC0002F7004E094F83C00FDF798FA0746DFF8ED
:104ED00080B140F68C2A0BF1180B062F47D294F8BC
:104EE0003800B8423ED03846FDF70CFA2078C007AB
:104EF00016D094F83A0094F8391000F00302914269
:104F000006D0A17A00F0010001F00101884215D11C
:104F1000FDF762FBFBF778FFFDF78AFC384689E076
:104F2000FDF75AFBFBF770FFFDF782FC3846FDF7F3
:104F300073FB207840F00100207099E7288820F06A
:104F400008002880206B810801EBD000504515D265
:104F5000B8F800100844ABF80000308840F00800B2
:104F600003E00DE0308820F00800308080E7B9F8D9
:104F7000001041F00101A9F80010DFE75046E7E713
:104F80000007288831D520F008002880308820F0DC
:104F900008003080FFF708F884F83C00FDF7B4FB08
:104FA000387820F0020038702078400604D5FEF7EB
:104FB000B3FA97F82F5004E094F83C00FDF71EFA7E
:104FC0000546062D08D294F83800A842B5D0FDF762
:104FD00003FBFBF719FF2AE02048C18841F040019C
:104FE000C180BDE8F05FFDF703BCC006288825D569
:104FF00020F010002880308820F01000308097F8D2
:1050000038000C2802D2401C87F83800387840F06D
:1050100002003870FEF780FA97F82F50787884F8FD
:10502000390094F83800A84287D0FDF7D5FAFDF78B
:10503000FFFB2846BDE8F05FFDF7EEBA4EF2BE1169
:105040000840288014E700001004004000040040DD
:10505000240400403C0100203C040020080A0020F9
:105060002DE9F04F514F85B0388820F0010038808D
:105070004E480026103006804D4CDFF838A14FF026
:10508000010894F85C0042F63029C10774D072B66A
:105090004948816941F400718161816941F480610D
:1050A00081614FF40040FEF7E5FE444D00212846A3
:1050B000FBF708FC00212846FBF7FAFBDFF800B1FC
:1050C00000215846FBF7F4FB00213E48FCF784FA28
:1050D0002846FBF713FD5846FBF710FD4FF4602000
:1050E000CDE902068DF8056000968DF810808DF8E8
:1050F000048069462846FBF793FD01231A460F21D9
:105100002846FBF7DEFD01212846FBF7D1FB0020F6
:105110004946401C80B28842FBD328462E600121BC
:10512000FBF70EFE28688007FCD524484C30006849
:1051300094F85C1021F001012144A1F85000FBF724
:10514000CBFB62B6FEF7F4F847F69061AAF80010C0
:1051500094F85C00401CC0B284F85C000C2822D299
:1051600012491431A1F80080388840F001003880DD
:1051700005B0BDE8F08FFFE7134920F00100085AA1
:1051800012490880114945F65800083908800F482F
:1051900047F25801001F01800C4920200C3908807B
:1051A000AAF80090D4E70320A070E1E700080040CF
:1051B0003C0400202C080040001002400024014064
:1051C0000028014008000240B8890008202C014056
:1051D0000029018802D041F0800101E021F0800126
:1051E0000180704710B50A884B88CC881A438B8899
:1051F00023431A430B891A434B8989891A430A436B
:10520000A0F8442010BD0021018041808180C18030
:1052100001814181818170470029818802D041F05C
:10522000010101E021F0010181807047002901881E
:1052300002D041F0010101E021F00101018070473D
:10524000002930F8441F02D041F4004101E0C1F3CD
:105250000E010180704700004B4910B5884202D111
:105260000121C41486E0B0F1804F09D0474988423B
:105270000DD101210220FEF71FFE0021022064E073
:1052800001210846FEF718FE002101205DE040499B
:10529000884206D101210420FEF70EFE00210420E1
:1052A00053E03C49884206D101210820FEF704FE64
:1052B0000021082049E03849884206D10121102008
:1052C000FEF7FAFD002110203FE03449884206D164
:1052D00001212020FEF7F0FD0021202035E030499B
:1052E000884202D10121441444E02E49884202D16F
:1052F0000121CC043EE02C49884202D101210C0559
:1053000038E02A49884202D101214C0532E028497F
:10531000884206D101214020FEF7CEFD0021402029
:1053200013E02449884206D101218020FEF7C4FD04
:105330000021802009E0204988420AD184150121FA
:105340002046FEF7B9FD00212046BDE81040FEF7DB
:10535000B3BD1A49884202D101210C040AE0184960
:10536000884202D101214C0404E0164988420AD146
:1053700001218C042046FEF7B7FD2046BDE8104011
:105380000021FEF7B1BD10BD002C0140000400401B
:1053900000080040000C00400010004000140040D5
:1053A00000340140004C01400050014000540140D5
:1053B00000180040001C0040002000400040014058
:1053C0000044014000480140002A828901D00A437C
:1053D00000E08A438281704730B5028C22F00102DE
:1053E0000284028C8388048B22F0020224F073056D
:1053F0000C882C430D8915434A882A43114DA84235
:105400000BD0114DA84208D0104DA84205D0104D28
:10541000A84202D00F4DA8420DD122F008054A89BA
:1054200023F440732A4322F004058A882A438D8995
:105430001D43CB892B4383800483C98881860284E2
:1054400030BD0000002C014000340140004001400C
:105450000044014000480140028B22F008020A4348
:105460000283704770B5028C22F010020284028C15
:105470008488038B0D8823F4E6464FF6FF7303EA16
:10548000052535430E8922F0200203EA061616434D
:105490004A8803EA02123243104EB04202D0104E44
:1054A000B04215D122F080064A8924F4406403EA10
:1054B0000212324322F040068A8803EA0212324383
:1054C0008E8903EA86062643CC8903EA84043443A2
:1054D00084800583C9880187028470BD002C014047
:1054E00000340140028B4FF6FF7322F4006203EA9E
:1054F000012111430183704770B5028C22F4807240
:105500000284028C8488838B0D8823F073031D43EF
:1055100022F400730E894FF6FF7202EA06261E433C
:105520004B8802EA03233343104EB04202D0104EA0
:10553000B04215D123F400664B8924F4405402EAAA
:105540000323334323F480668B8802EA0323334327
:105550008E8902EA06162643CC8902EA04143443F3
:1055600084808583C9888187038470BD002C0140B5
:1055700000340140828B22F008020A438283704784
:1055800070B5028C22F480520284048C8288838B52
:105590000D8823F4E6464FF6FF7303EA05253543ED
:1055A00024F400560C8903EA043434434E8803EA99
:1055B00006362643094CA04202D0094CA04205D130
:1055C00022F480448A8903EA8212224382808583FE
:1055D000C988A0F84010068470BD0000002C01406E
:1055E00000340140828B4FF6FF7322F4006203EA1D
:1055F000012111438183704701858282704782882F
:1056000022F07002828082880A4382807047A0F86C
:105610004010704730B502881B4B1C4C98420DD08F
:10562000A0420BD0B0F1804F08D0194DA84205D050
:10563000184DA84202D0184DA84203D122F070059F
:105640004A882A43154DA84206D0154DA84203D0DA
:1056500022F44075CA882A4302808A8882850A8893
:10566000028598420AD0A04208D00E4A904205D046
:105670000D4A904202D00D4A904201D1097A01862A
:105680000121818230BD0000002C01400034014026
:105690000004004000080040000C004000100040E2
:1056A0000014004000400140004401400048014017
:1056B0004FF6FF71818000210180C180418001721D
:1056C00070470029018802D041F0020101E021F079
:1056D0000201018070470029018802D041F00401D5
:1056E00001E021F00401018070470000204810B55E
:1056F00090F82010026801F01F001E4951F82000A8
:105700001D490242086802D040F4803001E020F4D4
:105710008030086019484FF000028079410618482F
:1057200024D4184903880C88E31A9CB201230F2C57
:1057300008D30C8804808468042C03DD124C247880
:10574000022C05D0427F012A06D00988418010BD75
:105750004377C2770A88428042880988891A89B2C9
:1057600040F21A629142F2D3C37710BD427710BD66
:10577000CC050020FC8D000898020020080A0020BB
:10578000240C0020F8060020EF0600202DE9F04F41
:10579000DFF8B8B16A48DFF8AC91DFF8ACA190F857
:1057A0000EC0BBF91A70BBF91C60BBF91850BBF9ED
:1057B0006C10BCF1070F48D2DFE80CF08D041A30F2
:1057C000485E7600D9F800208284DAF80020C2848E
:1057D000828CC38CA7EB820212B2A6EB83034A43EE
:1057E0001BB2594342F3CF2241F3CF23D11870E0CB
:1057F000D9F800204284DAF80020C284428CA5EB5C
:10580000820213B2C28C4B43A6EB820212B243F364
:10581000CF24514341F3CF23E11814E0D9F80020FD
:10582000C284DAF800204284C28C438CA6EB820248
:1058300012B2A5EB83031CB24A43614342F3CF2368
:1058400041F3CF24191949420AB244E0D9F80020A3
:105850008284DAF800204284828C438CA7EB820297
:1058600012B2A5EB83034A431BB2594342F3CF2242
:1058700041F3CF24111914E0D9F800204284DAF85A
:1058800000208284428C838CA5EB820212B2A7EBAB
:1058900083034A431BB242F3CF24594341F3CF223F
:1058A000A11849420BB216E0D9F80020C284DAF8F8
:1058B00000208284C28C838CA6EB820212B2A7EBFA
:1058C00083031CB24A4342F3CF23614341F3CF2207
:1058D000991849420CB2BBF91E50594605F21E56A2
:1058E000A64201DACE8306E0A5F21E55A54201DDEF
:1058F000CD8300E0CC83B1F9204004F21E559542DF
:1059000001DA0D8406E0A4F21E54944201DD0C84F9
:1059100000E00A84B1F9222002F21E549C4202DA0D
:10592000ABF8224008E0A2F21E529A4202DDABF828
:10593000222001E0ABF82230417B8173BDE8F08F7B
:10594000980200203C2401403C2801401C05002016
:105950002DE9F04704465748584D0026027856482E
:10596000022AB0F9301004D0082A7DD0092A07D0C5
:1059700008E0C27B022A02D1B0F8402032B1E187B0
:1059800069812E8184F83C60BDE8F0874C49DFF8DE
:105990003481496A0F14E7808068410210D5B4F958
:1059A000020040F2DA21884269DD40F26A41884211
:1059B0003FDCA0F2DA20FAF732FD0022424B4BE046
:1059C000C0F3C001C0F30020DFF8009181420CD188
:1059D000D8F8440040F2BA41884250DD40F66A11DE
:1059E000884226DCA0F2BA4032E039480078C0068E
:1059F0000CD5D8F8440041F2243188423FDD41F211
:105A0000D471884215DC00F6DC401FE0314890F884
:105A10007010012903D090F86F0001282FD1B4F93C
:105A2000020041F6C811884229DD41F678618842BA
:105A30000ADD0823B4F93E101A460020FEF704FFE1
:105A4000E087002819DB1BE000F5C760A0F50050D7
:105A5000FAF7E5FC00224B46FAF74DFC0E22FAF766
:105A6000B9FCFAF713FD00E01FE000B2C0F580407A
:105A700078438013E087002F02DCE68700E0E787A9
:105A8000E08F154FE880D8F844107964A7F84C00EF
:105A900000F076FBB7F84E00688198F80A000028FD
:105AA000388F00D1404228816CE70C48B0F8700074
:105AB000688166E7EF060020980200206000002061
:105AC0001C0500203C0100200000794000C09240ED
:105AD000D00600205C0C0020AC0800201C0A00202E
:105AE0002DE9F041B1F9025000232B241522854203
:105AF00003DAB1F90000BDE8F081B1F9AE5085429A
:105B000002DDB1F9AC00F6E701EB8205B5F9025010
:105B1000854201DD134600E01446E21852085D1C80
:105B2000AA42F1D101EB8206B6F90230834206DACD
:105B300036F9025C36F9044C31F9221006E01D46B4
:105B400031F92240B6F90630B6F90410401B091BA2
:105B5000C6178911B60346EA90468703A1FB070CD6
:105B6000CA1702FB07C201FB06215A1BD317FAF71B
:105B7000DBFA000A40EA0160001900B2B0F5804F7C
:105B8000B9DB43F6FF70B6E770B5134C40F224451D
:105B90002946204600F03EF800281BD0204600F0A1
:105BA000C7F82946204600F01DF80C4C002120467D
:105BB000FBF712FD2046FBF78DFDC0F1640008499C
:105BC000C0B20428087201D900F046F9BDE870405F
:105BD000FBF7C6BD70BD0000003801405800024010
:105BE000580600200A0A01219140C94301807047EC
:105BF0000029818902D041F4005101E021F40051D3
:105C000081817047002A828A01D00A4300E08A43DA
:105C10008282704730B501F01F0201240025C1F3D4
:105C2000421304FA02F2012B0FD0022B0FD0838A09
:105C30004FEA11210088134204FA01F400EA04003B
:105C400001D000B10125284630BD8389F0E7038AE1
:105C5000EEE710B5C1F3421301F01F040121A1408A
:105C6000012B07D0022B07D01430002A026805D080
:105C70000A4304E00C30F8E71030F6E78A4302608C
:105C800010BD000030B50446008A85B00D464CF6C4
:105C9000FF710840E98801432182A1894EF6F31083
:105CA0000140A8882A8910436A890A431043A081C9
:105CB000A08A4FF6FF410840A9890143A1826846A6
:105CC000FEF71EF91948844201D1039800E00298BA
:105CD000A189090400EBC00101EB0010296801D57E
:105CE000490000E08900B0FBF1F06422B0FBF2F162
:105CF00009010B096FF018056B4300EB8300A389C2
:105D00001D044FF0320306D503EBC000B0FBF2F0E8
:105D100000F0070005E003EB0010B0FBF2F000F02C
:105D20000F000843208105B030BD0000003801405D
:105D30008088C0F308007047F8B501210920FEF7FC
:105D4000C7F801218803FEF7C3F810258DF803502A
:105D50002020ADF800001A4E03248DF80240694659
:105D60003046FCF741FA16490C31086820F0200053
:105D7000086018208DF803004020ADF800008DF871
:105D8000024069463046FCF72FFA48208DF80300A0
:105D90008020ADF8000069463046FCF725FA8DF802
:105DA00003502801ADF800008DF8024069463046E6
:105DB000FCF71AFA01210420FCF768FAF8BD00008C
:105DC000000C014030B585B0FFF7B6FF00244FF45A
:105DD000E1300090ADF808400C201D4DADF80440B6
:105DE000ADF80A00ADF80640ADF80C40694628460B
:105DF000FFF748FF25208DF8100004208DF81100D2
:105E00008DF8124001208DF8130004A8FDF720FD45
:105E1000012240F224412846FFF71BFF01212846BA
:105E2000FFF7E6FEFBF7C6FC012280212846FFF7BC
:105E3000E9FE012240212846FFF7E4FE012202216B
:105E40000448FBF75BFCFBF7B5FC05B030BD000078
:105E5000003801404400024070B51D4D00242878F0
:105E6000432834D16878462831D1A878502807D003
:105E7000512805D0812803D0892801D0212826D196
:105E8000144E7071E9787172A81C891CFBF78CF8AC
:105E9000B072717A294409793182884217D106F1AA
:105EA0000E00017841F0020101700B48016841F0D9
:105EB00020010160317A0948002204E02B5D03557E
:105EC0002A55641CE4B28C42F8D38078707170BD9E
:105ED00084070020580600200C0C01408E0B002087
:105EE00070B51D20FDF793FCFDF716FB1D20FDF797
:105EF000A4FC154890F82F10144D0623144C85F877
:105F0000381090F83B1095F83B201143012A04D03B
:105F1000022A07D0042A0AD010E0827A8A420DD0E1
:105F2000007B09E0027D8A4208D0807D04E0827F08
:105F30008A4203D090F82000884200D123700020CC
:105F400085F8400070BD00003C0400203C010020AA
:105F5000EF0600200B4800214180A0F1B0018A89A2
:105F60008280CB891A44C2800B8A1A4402814B8AF0
:105F70001A444281898A1144818143F6FF71C181AB
:105F800070470000EC010020084940F61C72B1F98E
:105F90000C00904202DA00F59F7005E041F2E30246
:105FA000904201DDA0F59F70C8817047600000201D
:105FB00038B51348C16941F00401C1611E208DF854
:105FC000000002208DF801008DF8020001248DF8F8
:105FD00003406846FDF73CFC0A49842008800949D3
:105FE00047F690602C3108800020091F0880054981
:105FF00014310C80091F0880081F048038BD000080
:10600000001002400008004030B420491E4A457884
:106010008B7A114692F83B4091F83910AC4218D176
:106020004BB10379994202D04379994201D1407929
:106030001AE0807909E08379994202D0C479A142BB
:1060400002D182F82F3011E0407982F82F0030BC65
:106050007047C578AC42FAD16BB1C379994202D08E
:10606000037A994205D1007A82F82F0030BCFEF7FE
:1060700081BC407AE9E7437A9942E2D00479A142AF
:10608000DFD0007AE1E700003C0400203C01002062
:10609000FEE700002DE9F0470446007F012868D1A3
:1060A0003548E1880288511A89B2072916D3008839
:1060B000E080B4F9000044F2DD414843401346F665
:1060C000D96148438013A060401000B2A0814FF016
:1060D0008051B1FBF0F0FAF79DF92061B4F90C6042
:1060E00096B1B4F902104DF6B05048430014A082A6
:1060F000B4F904704DF6B05207FB02F24FEA2245A4
:10610000E58204D4024603E00020E08330E042420E
:1061100012B22283002D01DB2B4600E06B421BB242
:10612000DFF85890638398464FF4804AB24208DA09
:10613000FAF767F92169FAF73AF8FAF78EF9801356
:1061400004E0002901DA484600E05046E083B0450B
:1061500009DA2846FAF755F92169FAF728F8FAF723
:106160007CF9801304E0002F01DA484600E0504635
:106170002084BDE8F0870000F806002000C0FFFF83
:1061800010B52248234C01782148022905D1C17B52
:10619000022902D1B0F8401029B1008EA4F84E00B7
:1061A0000020208710BD90F846101A48B0F844002F
:1061B00000B239B318490978C1F3810101291BD014
:1061C00002291CD0154900BFFBF75AFE1149A4F85B
:1061D000400080B2483101F099FAB4F94C00B4F9AA
:1061E0004A2041425143891324F8381FB4F9101052
:1061F00048438013E08210BD0849D839E4E70749D5
:106200006C39E1E705496C31DEE70000EF0600205C
:1062100098020020AC080020B4040020E2870008A7
:106220000348002180F82A10C183018770470000CD
:10623000AC08002010B504000B462D4AC3F1000045
:1062400028D56442002B12DAA04207DA214600F07A
:1062500027FA32F81000C0F5404041E001462046E0
:1062600000F01EFA32F8100000F5004038E0A342BA
:1062700008DA2146184600F013FA32F8100000F54B
:1062800040402DE0204600F00BFA32F81000C0F537
:10629000803025E0002B12DAA04207DA214600F018
:1062A000FFF932F8100000F5804019E00146204661
:1062B00000F0F6F932F81000C0F5004010E0A342FB
:1062C00008DA2146184600F0EBF932F81000C0F564
:1062D000804005E053B1204600F0E2F932F81000AA
:1062E000B0F5004F01DDA0F5803010BD002010BDDD
:1062F000C489000840438013494300EBA1300022C9
:106300000302002B14DDB3F5001F01DC802001E047
:106310004FF4005093FBF0F1014401EBD1714910AF
:10632000814206D0521CD2B20846062AF2D300E0BF
:106330000021C80000B2704702E008C8121F08C15F
:10634000002AFAD170477047002001E001C1121FF6
:10635000002AFBD1704700002DE9F047A44CA54866
:1063600021880288511A89B20F297DD30088A4F1AF
:106370003C052080288F08B1401E28872B789E4A34
:10638000C3F3810001281DD0022820D0D18B98486A
:106390009A4FDFF86C92407E0026B1F5926F1DD8BF
:1063A000142819D378206076F88840F01000F8801F
:1063B00040F26660A88123F001002870D67389F846
:1063C000006015E0D08B00EB4000C00302E0D08BF2
:1063D0008C494843010CDAE7401C04E0B1F5DB6F5F
:1063E00006D310B1401E607602E043F00100287031
:1063F000B5F90200B5F914304143C3EBC303C1F34F
:106400008F31C3F3D10303EB510109B2A982904646
:10641000D28B4FF080535043B5F91620C0F38F3024
:10642000C2EBC202C2F3D10202EB500000B2E8821A
:10643000AA6A42431213EA6293FBF2F22A63724A97
:106440001080A2680A44A260E1680144E160207CF7
:10645000401CC0B22074072806D942F3CF0028831D
:10646000C9106983E66000E0BFE0A66041F6C8019C
:106470002674884204DD298B644AB2FBF1F1E9817C
:10648000C117890341EA9041800342F69B420023F1
:10649000F9F74AFEA88456482A78A0F13C005C49E6
:1064A000B0F90600930700FB01F14FEA2141C2F366
:1064B000810215D5012A07D0022A0BD04FF268516C
:1064C00041430914A18011E049F68C425043001465
:1064D000A0801FE04CF6183141430914A18025E04B
:1064E000012A0DD0022A17D0A08069844949484367
:1064F0000014E083FBF7E4FA47480088C0B143E0AA
:106500004AF65C3242431214A2804BF62C225043CE
:1065100000146884E183EDE74DF2AC514143091466
:10652000A1804EF27C414143091469843B49DEE776
:1065300095F8200000BB88F80F6089F80060B5F975
:106540001A00A0F50C519F39B1F56E7F18D8617F04
:10655000F42912D93249E8802E4AA1F84600504366
:106560000014A880A1F84400FF2085F8200081F8DD
:1065700028002C493C20087006E0491C617703E0A4
:10658000607F08B1401E6077B5F91A10B4F91E009B
:1065900081420EDDA07E7D2809D9F88840F00800F0
:1065A000F8802148017821F0020101700EE0401CC2
:1065B00006E0A0F23D10814208DAA07E10B1401E34
:1065C000A07603E0F88820F00800F880B5F91810EC
:1065D000606908446061217E491CC9B221761F2987
:1065E00003D94011A88366612676BDE8F0870000D4
:1065F000F0040020F806002098020020080A00207D
:10660000EF06002030330100BC09002074E8260B9F
:10661000CC0E010048850100FA060020D04501009B
:106620005C0C0020EC060020C6050020024941F663
:106630008B30886270470000B404002070B5164C9F
:1066400006252078062825D2DFE800F003080E147E
:106650001A211248FAF7E6FC012016E00F48801DC7
:10666000FAF7E0FC022010E00C480C30FAF7DAFCF4
:1066700003200AE009481230FAF7D4FC042004E0B1
:1066800006481830FAF7CEFC0520207070BDFAF7E6
:10669000E9FC2570257070BDF0060020BA8800085E
:1066A000090A05D0B0FBF1F0FF2800D9FF207047A0
:1066B00000207047D0E90021C368521A5A4301EB09
:1066C000A231816041607047B0F90020B0F902103A
:1066D000B0F90630521A5A4301EBA2318180418051
:1066E00070470000F0B54F4C20884F49504E514B39
:1066F0008A89801A82B24D480F2A057801F14C0030
:1067000032D322888A81197A5FEA017C0146B1F985
:10671000021001F1020217B2A1F1020212B20BD56E
:10672000022D01D044490FE0DFF810C1BCF900C0D0
:10673000614513DC17DB13E0022D15D1D6F844C0F8
:10674000BCF5FA5F03DC3E49098841800CE0DFF8C4
:10675000F4C0BCF900C0614505DB01DD428003E007
:10676000A0F802C000E04780018F2288A2EB01015F
:1067700089B29C2941D321880187996A0022B1F509
:10678000804F2CDBB16CB1F5405F28DD2E4940F223
:106790006664B1F91010A14211DD43F69914A142CB
:1067A00002DB40F2333108E040F23334A1F266619B
:1067B000614343F2333491FBF4F1818700E0828737
:1067C0002249B3F806410978C1F381011CB1818FD8
:1067D00001F21E5119E093F84630022B0ED0828749
:1067E000022D00D08287B0F95410B0F93C2001F19D
:1067F000140393420BDAA0F85430F0BD012901D004
:106800000229E4D1818F01F233318187E8E702F177
:106810001403994203DD1439A0F85410F0BDA0F818
:106820005420F0BDF806002014000020EF060020E0
:106830003C01002098020020B2040020B004002097
:10684000AE040020AC0400201C050020B40400208D
:106850002DE9FC4101210220FDF722FB0121192035
:10686000FDF736FB01213C48FBF710FD4027ADF852
:10687000007003248DF802400420384D8DF8030089
:1068800069462846FBF7B0FCE001ADF800008DF842
:1068900002401C208DF8030069462846FBF7A4FC43
:1068A0004FF4E0712846FBF726FDA815ADF800006F
:1068B0008DF8024010208DF8030069462848FBF748
:1068C00093FC4FF4A060FCF7F5FF1D208DF8040049
:1068D00001268DF8056000258DF806508DF80760BB
:1068E00001A8FCF7B5FF1F498C2008801D494FF611
:1068F000FA702C3108806E20091F08801948143066
:106900000680184808300780164920310D80154A46
:10691000D020121D1080134A45F2F3001832108067
:106920000A1F45F2500010800E4A4FF6FF703832B1
:106930001080121D1080121D108041F21B10088063
:1069400000F012F8FBF754FF064810300580001FD6
:106950000480BDE8FC810000000C1A00001001401A
:10696000000C01400004004070B51D20FCF744FFFE
:106970002A4D40212846FBF7B5FC8400802128469B
:10698000FBF7B0FC44EA4004A9152846FBF7AAFC33
:106990000443E0B2224C84F83C00FBF72FFD05468F
:1069A000052805D91F48C18841F04001C18001E098
:1069B00084F838501C48007A000703D594F8380052
:1069C0001A490D5C4FF6FA702063E062A0626062C3
:1069D0002062E061A0611648606300206064A064EA
:1069E00084F83F0084F84000FBF7B6FCA07AFF284B
:1069F00011D0022084F83D000E4800882066284609
:106A0000FCF758F9207820F001002070BDE87040B4
:106A10001D20FCF707BF0120ECE70000001001403B
:106A20003C010020080A002098020020C8910008BC
:106A3000DCFF0500240400402DE9F0434E484F4997
:106A400002880B889A1A92B20F2A69D309880180AA
:106A50004B49098B027D00EB42029180017D491C6C
:106A6000C9B2017508295BD3002404752246017D53
:106A700000EB4103491CB3F90430C9B202EB6302D5
:106A800012B201750829F2D33E4904753E4B4A8083
:106A900044800E789D895FEAC67C40F638694FF0E5
:106AA000030714D0A2F22B5C42F6E858C44520D369
:106AB000A1F1020C26F00204ACF8002047750C701E
:106AC00040F22B54A24211DA45F004021EE046F0D7
:106AD00001060E704A4507DD45F001029A8126F055
:106AE00002020A70477519E0447517E045F002028A
:106AF0000CE04A450CDA8775427D12B1521E427590
:106B00000CE046F002020A7025F007029A8105E0C7
:106B1000B30703D5837D2BB15B1E837540888880C6
:106B2000BDE8F08342F6AA239A4222DAB1F9043092
:106B30002BB941F2CD05AA4201DA4480EEE7134CAD
:106B4000920302EB843241F67244B2FBF4F214B2C7
:106B500040F2333502464480AC4200DA5580B2F947
:106B60000240E41A04F5A374B4F5237FD6D8438019
:106B7000D4E74FF48043FAE7900A0020F80600209B
:106B800098020020C6050020080A0020C8F1FFFF77
:106B90002DE9F0416C4CDFF8B4E14FF0000594F8BA
:106BA0002810C80706D094F92C104B42002956DD56
:106BB0000E4655E0664884F82B50E586654A90F805
:106BC000380084F834001586CEF80450CEF808500A
:106BD000614E40F26663CEF80C50A4F8703036F87F
:106BE00010005E4E768830444FF6FF7606EA80004D
:106BF00024F8240B4FF080602060A3202084608460
:106C00005810A084E38440F69910208558006085D0
:106C10004FF48050A08541F23330E08541F2666048
:106C2000208641F69910608641F6CC40A0864FF44C
:106C30000050E08642F23330208742F2666060877F
:106C400042F69910A08742F6CC40E08782F89D502A
:106C500041F00100207184F84450BDE8F0811E46E7
:106C600094F92B004242002801DD074600E0174658
:106C7000F61B012E0BD0002800DB02465FFA82F6DD
:106C800084F82C0094F84300012805D041E0002945
:106C900000DA1946CEB2F3E794F92D305942002BB1
:106CA00001DB184600E0084694F92E20C7B2504296
:106CB000002A01DB944600E08446BC4508DD002A3A
:106CC00000DA0246D7B2002B00DA0B46D8B207E052
:106CD000002B00DA0B46DFB2002A00DB1046C0B200
:106CE00004EB4000B0F9441004EB470030F9442FA6
:106CF00011444910018084F8435084F8325084F8DC
:106D0000315084F8305084F82F5084F82E5084F895
:106D10002D5004EB46007546B0F94400E086BEF8FD
:106D20000410C82309B26422FDF78EFD6860E9688B
:106D3000401AA9680844A860B5F900104843C01378
:106D4000E860A4F8700088E71C0A0020B405002061
:106D50003C01002098020020DA9100086000002029
:106D60002DE9F0415F4C94F82800C00779D05E48C7
:106D700094F83410002690F838005C4D814271D0B0
:106D80005B4AA4F866605B4F535C2246834292F9EB
:106D90002B2002D07B5C83420FD1521C52B284F86C
:106DA0002B20795C814202D1521C84F82B2094F96B
:106DB0002B100F291BDD0F2117E04F4B5F5C4F4B52
:106DC000874202D05F5C874211D1521E52B284F8D2
:106DD0002B20595C814202D1521E84F82B2094F959
:106DE0002B206FF00E018A4201DA84F82B103D4906
:106DF00094F833302D3194F82B205A5494F83310F2
:106E0000491CC9B284F83310062901D384F83360D1
:106E100094F92D2094F92F108A4211D194F9312040
:106E200091420DD194F92E2094F930108A4207D165
:106E300094F93220914203D1012184F8431001E0FA
:106E400084F84360284984F8340094F92B30097899
:106E5000012B0DDD254A4F07926804D542F0080248
:106E600003E03CE015E022F00802AA6084F8290063
:106E7000B3F1FF3F0ADA4907A96802D521F00801FA
:106E800001E041F00801A96084F82900FBF764FAE9
:106E900011E094F8430001280DD1B4F8660043F6E0
:106EA0000951401C80B2A4F86600884203D9A4F8B6
:106EB000666084F84360E87B082810D0B5F930108C
:106EC000512341220020FDF7BFFC2886002806D16F
:106ED0000B48067014F8280F20F001002070BDE860
:106EE000F08100001C0A00203C01002098020020D4
:106EF000BC910008C2910008CE910008D49100080E
:106F0000EF06002030B52049204AB1F86A301088D9
:106F1000C01A80B20F2836D31088A1F86A001C4D21
:106F200000204FF000432A5C940903D00124B4EB05
:106F3000921F24D1D20622D0164A52F8202012687D
:106F4000134C123434F81040224201EB000494F93F
:106F5000722008D00A2A04DB0A6823FA00F42243CC
:106F600008E0521C09E012F10A0F05DC0A6823FA56
:106F700000F4A2430A6002E0521E84F87220401C12
:106F8000C0B21128CFD330BDCC050020F8060020B8
:106F9000C88D0008C88E00082DE9F00779497A48A5
:106FA0000A8903889A1A92B2082A74D30088088141
:106FB000A1F12C0042890AB1521E4281734A92F813
:106FC0002820802A67D302F03F020A70C2890AB1E2
:106FD000521EC281B1F90620902A0CDB8A46FF2A94
:106FE00009D08146C089002855D16948002300781E
:106FF000092805D005E0BDE8F007624800F096B921
:107000000823644A92F8EA500DB143F00403624841
:10701000817AC90701D043F00203D2F808C05FEAC1
:107020000C5101D543F00103176800215B4EFC03AE
:1070300002D596F8654004B18021C4885FEA4468AF
:1070400001D541F040015FEA845801D541F02001AB
:107050005FEAC47801D041F01001007A400701D501
:1070600041F008014E480078C00701D041F004010A
:10707000A00601D541F001010020012D00D108201A
:1070800096F8705085B992F84620022A04D0012A59
:1070900005D03AB108E072E040F0030004E040F0AF
:1070A000020001E040F001007A0701D440F0200026
:1070B000CCF3C0020025CCF3002C624502D13A0784
:1070C00000D4042596F86F20012A01D145F001056E
:1070D000344A0027BC4612783E46C2F38102012A98
:1070E00004D0022A04D0032A04D004E0022602E0DD
:1070F000042600E010262C4A64060ED5214C1C34D0
:107100002478240609D51478640606D4274A40F664
:10711000CC44926D6243140C05E0B2F8AE2040F608
:1071200099146243940B4FF008088AF80A804FF0D4
:1071300061088AF80B808AF80C308AF80D108AF8FA
:107140000E008AF80F508AF81070270A4B4083F01F
:107150006901414069408AF8117079408AF812400B
:10716000614052468AF813C071408AF81460517524
:107170004FF4C871A9F80E10FF20AAF80600BDE868
:10718000F0077047B4060020F8060020CC05002068
:10719000EF06002098020020080A00205C0C002066
:1071A00000090020B40400203C010020E807002072
:1071B0004E48816941F0FC0181614FF4A060FCF709
:1071C00079FBFBF7A3FBFCF7E1FCF9F7EFFCFCF71D
:1071D000CFFAFDF73FFAFFF73BFBFCF70FFAFFF79B
:1071E000C3FBFBF705FB424D4FF40050A5F8160119
:1071F000FEF7E8FD00214FF4FA5340F2EE220020A2
:10720000401C80B29842FBD3491C89B29142F6D30C
:107210003848002680F87260F9F75EFBF9F7F8FF4E
:10722000FCF7E4FCF9F7CCFEFEF7C2FE102232496F
:107230003248F8F7AAFF324C334FE08820F0400084
:10724000E0803048017821F020010170FA20F881B7
:107250004FF49670E887FFF7E9F92C492C48FCF7C2
:107260003BFC2C48FCF764FC2B48416A88472B48C0
:10727000416B8847FEF7D4FF2948FAF71CFC2949DF
:107280004220C8802849C8603E71E088E08120899A
:10729000208260896082FAF71FFFFAF781FEFFF70C
:1072A0005BF8FFF7C9FB00F0F9F9FFF72BFE00F0E0
:1072B0009FFFFEF71BFAFAF7D3FCFBF719FDFFF768
:1072C00011FAFCF7EBFEFBF73BF9FBF76DF900F069
:1072D0007BF8FFF761FE1248FAF7B6FA00F070FA91
:1072E000FDF7FCF9FAF71EFCCFE7000000100240A2
:1072F000980200201C0500205C0C00200C060020D9
:10730000080A00203C010020EC060020880800202C
:1073100064080020F803002034000020D000002082
:10732000880900201407002028040020F0B5234914
:107330000278B0F9064000231F4E31F81210FF2CDE
:1073400018D0B0F904701E4DBC4231DA00EBE407EE
:1073500004F00704BF7AA7408478FFB23CB190F8EC
:1073600001C0ACF1010C64451FDA3C061DD455F890
:1073700022200DE056F82220116012498A79521C11
:10738000D2B28A71022A02D38370C3808B71F0BD9E
:1073900011608178491CC9B2817042789142F6D35C
:1073A0008370C188491CC180F0BD56F82220EFE7E8
:1073B00055F822201160F4E7A88F0008DA8D000844
:1073C000508F000888060020F0B561486149B0F888
:1073D0006C200B889A1A92B29C2A7BD30988A0F859
:1073E0006C105D495D4F91F82A1001F0070297F883
:1073F0004610022A00D1491E594C80F83E104FF029
:107400000203E2884FF00001550401D5012236E065
:10741000A489E50601D5062231E0250701D5082219
:107420002DE0550603D44F4D2D78AD0601D504222D
:1074300025E0150501D5072221E0150601D50A2210
:107440001DE0950601D50C2219E0150701D50B2288
:1074500015E0550701D4D50501D510220FE0D5065A
:1074600001D505220BE0650703D4A50701D4E40785
:1074700002D080F86E3007E0920403D5032280F832
:107480006E2001E080F86E10374A384C92F820E008
:10749000324A251FD2F808C02D4AB2F87060721C1B
:1074A00092B2BEF1000F0DD02CF4000CC7F808C04A
:1074B00090F86E70B7B11E2F1AD090F86F200AB3F3
:1074C00025E007E04CF40006BE60A0F870200A2A10
:1074D00001D22360F0BD142A01D22B60F0BDA0F8C8
:1074E0007010F0BD2B60A0F8701080F86F10F0BD28
:1074F000642E04D2A0F87020322AEED3E9E7A0F877
:107500007010EAE77F1C80F86F70A0F8701090F898
:107510006F20012A10D0002AE9D0B0F87060761CE4
:10752000B6B2A0F870601E2ED7D323603C2EDED9F1
:10753000521E80F86F20D2E7B0F87020521C92B231
:10754000A0F870202360C82AD1D980F86F10C6E750
:10755000CC050020F80600205C0C002098020020DA
:10756000080A00203C010020B4040020141C014043
:10757000F0B54248B0F84810491C89B2A0F848104C
:1075800002297AD33E490024A0F848400A783D4BAE
:10759000042A57D04FF48041082A0BD0A0F10C02E6
:1075A000B2F900208A4200DA1146B3F980208A42FB
:1075B00000DA1146344A92698A4200DA11B24182F5
:1075C00082881D8AC2EB8502304D12B22D78C5F338
:1075D00081062A4D42F2AA467243B5F976509212BC
:1075E0006A431213C26086681546C6EBC60642F3AC
:1075F000D102F60202EBA6328260C66C1644C66463
:10760000B0F850707F1CBFB2A0F85070B7F5806F13
:1076100004D3B6120682A0F85040C464891A1C4EE6
:10762000C26A724340F255564E4302EB4602466A26
:1076300032444262B3F93030B2EB034F06DD1A0434
:10764000426206E01349B1F90410B3E7002A00DAF8
:107650004462C162104990F83D2091F838108A4286
:107660000BD080F83D10B0F84210A0F84410B0F8EC
:107670004010A0F84210A0F84050F0BD1C050020BA
:10768000EF06002098020020F40B0020B404002034
:10769000C3F5FFFF100C00203C01002017481849DB
:1076A000B0F85A200B889A1A92B20F2A25D309886B
:1076B000A0F85A10134941F6302391F84D10CA072B
:1076C00001464FF48042B1F9001059438913A0F8E4
:1076D0006C100D490B78A0F10C01022B06D1B1F909
:1076E0000030934202DA1B1D0B8000E00A8000216B
:1076F000A0F8601020F85C1F428070471C05002035
:10770000F80600205C0C0020EF0600204FF6FF7208
:1077100002EA800210F4404315480ED0B3F5804FC2
:1077200014D0B3F5004F4FEA122216D0C2F5807381
:1077300030F813305B424B8005E0120A30F812300B
:107740004B80C2F5807230F812000FE0120AC2F5C9
:10775000807330F813304B8005E030F81230C2F5FA
:1077600080725B424B8030F81200404208807047C4
:10777000C48B0008104A518A908AD28A163846393A
:10778000A2F1110200D54942002A00DA5242114406
:10779000002800DA40420844084943F6284300B272
:1077A000B1F936205A43921340F2D733584302EBD3
:1077B000A030C88670470000980200201C050020F9
:1077C000F0B5904990480A8903889A1A92B23E2AE5
:1077D0001ED30088088101F138004FF4FA63428A11
:1077E0009A4202D2521C428200E04382874A92F8B7
:1077F0002220802A0CD302F03F020A70B1F9062041
:10780000402A06DBFF2A04D0C2883AB1521EC28049
:10781000F0BDBDE8F0407B48FFF788BD428A9A4240
:10782000F6D307784FF0010E3A074FF0FF055BD50E
:10783000847A40F2DC52630708D444F00403837274
:10784000C28081F80BE081F80AE04CE04378072B16
:1078500005D0032B03D0052B01D0062B07D16606DC
:1078600005D444F040038372C280052239E0654AA2
:107870005FEA437C02F138024FF42076127A0DD58C
:107880005FEAC26C0AD45FEA446C07D442F010028B
:1078900002723A0628D4C680192222E0DF0709D0F6
:1078A000970707D4670605D442F002020272C68029
:1078B000042216E09F0709D5170707D4670605D4E9
:1078C00042F008020272C68003220AE01B070BD5B1
:1078D000530709D4630607D442F004020272C6803B
:1078E0000B22CA728A72CD80494AB2F92230B2F9AB
:1078F0001A7003F23D140022A74200DB0276414ECB
:10790000444C06F13806A479B6895FEAC46C06F1E6
:1079100001064FF4C874B6B213D58681B6F57A7FE6
:1079200005D9017A21F0800101728281F0BD037ACC
:107930001E06FBD4828143F080020272C4801120B3
:1079400035E09F4216DA037E052B13D28681B6F509
:10795000487F04D98281027A22F040020272027AC0
:107960005606E3D45B1C037642F040020272C480E8
:1079700002201CE0284B1C89C4F3C006C4F3002776
:1079800040F2EE24BE4216D11E78360713D4427E52
:10799000012ACBD1428BB2F5167F02D2521C428310
:1079A000F0BD827A42F002028272C4800F20C87257
:1079B0008872CD80F0BD93F80D714FF40046012F11
:1079C00018D1164F41F6583C7F6C674512DD83F89D
:1079D0000CE1134B1E60C38AA34202D25B1CC3821C
:1079E000F0BD4FF4FA73C3801C23CB728B72CD8031
:1079F000C282F0BDC2820A4883F80C21001F0660D3
:107A0000F0BD000098060020F8060020CC050020FC
:107A1000B4040020080A0020980200203C01002045
:107A2000140801402DE9F05FF848F949DFF8E4A3B4
:107A3000007E0A1D131D0128504650D030F85A4FC1
:107A40000C8041881180BAF85E001880FDF79EFE18
:107A5000F14DF24C49F2CD32B5F91E006083B5F913
:107A6000201043F6CC4C00EB410151430914A18393
:107A7000B4F92230B4F9206001FB03F200FB0622C6
:107A800042F38F326282B4F91670714307FB0CF730
:107A9000BF1340F2333C02FB0CF200FB131007EB68
:107AA000A232E2828013A082DD48DE4E406C30605C
:107AB000316930468847DC49308948800846FDF7FF
:107AC00047FFDA4F01264FF0000B3878A4F14C093C
:107AD00008280CD0618E218204284AD01AE030F8A0
:107AE000604F0C8041881180BAF86400ADE7D0483F
:107AF00090F92B10491C022939D890F8681019B157
:107B0000B4F85200208205E0618E2182A4F8521060
:107B100080F86860B4F91410B4F90A00C54AF9F79E
:107B2000B1FCE062BAF91611884204DDC148E16295
:107B3000027A9140016299F800C0BF494A4644F672
:107B40003D2849F27A40BCF1000F2ED0BCF1010F64
:107B500043D089F800B0387804280DD0B54AB4F97C
:107B60001610B4F90800243AF9F78CFC08E0608E8E
:107B7000C8E7686A0014E062A948807AF0B3AF48A9
:107B8000AF4DA0622860E06A68602846FCF7ECF818
:107B9000A84F287C383F01284AD0A06A3860A948FD
:107BA0000178C90748D0406947E0B5F91EC0C44410
:107BB000844509D8B5F920C0C444844504D8B5F932
:107BC000225045448542C6D982F801B089F8026046
:107BD0008AF80FB087F800B01BE089F800B0B5F95B
:107BE0001E20DC46424482420BD8B5F92020424494
:107BF000824206D8B5F92220424400E015E08242D4
:107C00000ED989F8026089F801C08AF80FC087F898
:107C100000C0C88840F40060C880FAF7B3F99AE75A
:107C2000C88820F40060C88095E74FF4AF70A7E7DC
:107C300068693860A86900E0E06A78607D48383893
:107C4000FCF706FA754D754935F8100F3C39FFF70A
:107C50005DFDD9F81010C9F86C10B5F91010B868AE
:107C6000B5F9122000FB01F4FB68504303FB1244FA
:107C700044F38F3703FB010040F38F34DFF8C881F2
:107C8000AF86EC86A8F802704546A8F80440404646
:107C9000FEF700FA287F614D383D012830D0604260
:107CA00041104DF6B350474369803A142A80484644
:107CB000A9F804408B18C380891AA9F808108AF81B
:107CC0000CB0B9F90430D84654464946002B00DDC3
:107CD0002673B1F90600002802DD227B921C227374
:107CE000B9F90820002A02DD217B091D2173217BBF
:107CF00007291BD2DFE801F01A162F142B182D00CC
:107D0000B8F920304DF6B352594249106980B8F99C
:107D10001E00504302142A804846A9F80430C9E7DF
:107D2000667303E0022100E003216173DFF8EC9049
:107D3000464E474F99F800100129617B0DD0072965
:107D400063D2DFE801F0E7FEFDFCFBFAF900042155
:107D5000EBE70521E9E70621E7E7072955D2DFE848
:107D600001F0D9041B3D7999AF0001461846FBF795
:107D700099FE2860B5F90200B5F9001043F20462DB
:107D800001445143090C5043A4F85A10000CA4F8C4
:107D90005C00A4F85E8027E1404201B2504200B28C
:107DA000FBF780FE2860B5F9020043F2046141430D
:107DB000090CA4F85A10B5F90010084443F2046104
:107DC0004843000CA4F85C00A4F85E803AE1304619
:107DD000F8F74AFF01231A46072190E0194610469A
:107DE000FBF760FE2860A4F85A80B5F90200B5F9E7
:107DF000001043F2046201445143090C5043A4F8BB
:107E00005C10000CA4F85E004BE183E088090020C0
:107E1000342C0140980200201C0500206000002046
:107E20003C01002028040020E8030020EF06002089
:107E30001C0A002088080020080A0020A2FEFFFF7C
:107E4000E009002000090020BC09002000240140B6
:107E5000002801405942404209B200B2FBF722FE1D
:107E60002860A4F85A80B5F9020043F20461414346
:107E7000090CA4F85C10B5F90010084443F2046141
:107E80004843000C39E13046F8F7EEFE01231A466C
:107E9000052134E01146FBF705FE2860B5F9020024
:107EA00043F204614143090CA4F85A10A4F85C8021
:107EB000B5F90010084443F204614843000C47E15F
:107EC000504201B2584200B2FBF7ECFD2860B5F910
:107ED0000200B5F9001043F2046201445143090C59
:107EE000A4F85A105043A4F85C80000CA4F85E007B
:107EF0005EE13046F8F7B8FE01231A4606213846FF
:107F0000F8F7B2FE01213046F8F724FE0121384689
:107F1000F8F720FEB34EB9F808004D463080B9F8A6
:107F20000A007080B9F81000B0803046F9F7D8FC2C
:107F3000B4F85A00F18805E018E1ECE0BDE08EE00D
:107F40005EE031E00844A4F86000B4F85C003189D8
:107F50000844A4F86200B4F85E0071890844A4F8EB
:107F60006400317EA048012978D034F85A1F01807E
:107F700061884180A18881809B49028808310A80FC
:107F800042884A80808888809748896A0830884774
:107F900095F8360000287DD0F9F764F815F8360F0B
:107FA000401E2870BDE8F09F01461846FBF77AFD99
:107FB0002860B5F9020040F681514843801368807B
:107FC000B5F9001040F68152514389134218A2F6C8
:107FD0008152524252082980A4F85E201044A4F82D
:107FE0005C000844A4F85A0000213046F8F7B2FDBE
:107FF00000213846F8F7AEFD01231A460621E6E6D1
:10800000404201B2504200B2FBF74CFD2860B5F986
:10801000020040F68151484381136980B5F90000A0
:1080200040F68152504380130A18A2F68152524200
:10803000520828801144A4F85E20A4F85A1008447D
:10804000A4F85C0000213046F8F784FD0021384692
:10805000F8F780FD01231A460521B8E6B4E0194679
:108060001046FBF71FFD2860B5F9020040F681516C
:10807000484380136880B5F9001040F6815251439F
:1080800089134218A2F68152524229805208A4F85C
:108090005A2000E09BE01044A4F85E000844A4F8D5
:1080A0005C0000213046F8F755FD00213846F8F70E
:1080B00051FD01231A460721E5E65942404209B223
:1080C00000B2FBF7EFFC2860B5F9020040F68151E1
:1080D000484380136880B5F9001040F6815251433F
:1080E00089134218A2F68152524252082980A4F8FC
:1080F0005A201044A4F85C000844A4F85E00002153
:108100003046F8F727FD00213846F8F723FD012314
:108110001A460621B7E61146FBF7C4FC2860B5F9FC
:10812000020040F68151484380136880B5F9001081
:1081300040F68152514389134218A2F681525242AD
:1081400052082980A4F85C201044A4F85A0008447E
:10815000A4F85E0000213046F8F7FCFC0021384608
:10816000F8F7F8FC01231A460521C2E6504201B295
:10817000584200B2FBF796FC2860B5F9020040F6C1
:108180008151484380136880B5F9001040F6815250
:10819000514389134218A2F6815252425208298053
:1081A000A4F85C201044A4F85E000844A4F85A0027
:1081B00000213046F8F7CEFC00213846F8F7CAFC1B
:1081C00001231A46072194E634F8601FCFE60748DA
:1081D0000088A0F5D04168393FF4E4AEBDE8F05F17
:1081E000F9F712BE880900202C000020182C01404D
:1081F0002DE9F041904C9148B4F85A100288511A78
:1082000089B20F296FD30088A4F85A008C480088DF
:10821000DFF83082C0074FF000054FF0010741D072
:10822000874AD4E90C1024321388B1EB530F02D2E1
:108230001288511A08444FF4F371884200D208465C
:108240008149B1FBF0F0616CC1F35101084406466D
:108250006064F8F7E4F800227C4BF8F74CF84FF034
:1082600040427B4BF8F747F80E22F8F7B3F8F8F7DF
:108270000DF9A4F8A40094F86500401CC0B284F87D
:108280006500082834D36C4898F84620001F03780E
:108290009A4201D0027045806E4A13786E4A23B12B
:1082A000458021E06564A56458E0D8F89410A1F5F4
:1082B000FA618E4211DD616D8B1C9E4205DDB0F9C5
:1082C00002100A290DDA491C06E08E4205DAB0F9DF
:1082D0000210002908DD491E4180B0F902000A2879
:1082E00002DB177001E0A2E01570666584F8655046
:1082F0005A484FF4A5420178C1F38101012949D0C0
:1083000002294AD044F687712181A4F8A020B0F94F
:10831000243089B24B439B13A4F89C30B0F90E0073
:1083200000237043B0FBF1F0A16CC0F3D100C1EBAE
:10833000C101C90200EB9130A064F017810341EA4A
:108340009641B003F7F7F0FEB4F8A210C1EBC101FB
:10835000C902C00800EB9130A4F8A200616CA06EC5
:108360000844A06694F86C20521CD2B284F86C20A9
:10837000082A05D3C008A4F86E0084F86C50A566DE
:10838000374A384ED388580633D498F80F0002285D
:1083900006D02CE043F20451B6E744F24621B3E79D
:1083A000B06840F69916B04221DD94F8380094F890
:1083B0008660B0420CD084F8860094F83D0000F04E
:1083C0000106C0F34000864202D1A4F8825004E0C6
:1083D000B4F88200B0F5966F05D2B4F88200401C64
:1083E000A4F8820005E043F08000D08001E0A4F80A
:1083F0008250114894F83F20B0300C2A01D2C57445
:1084000000E0C774174B41F2482641F2504C93F8F4
:108410003C400C4B0C2AB3F882300AD3B14208DB43
:10842000012C06D0614502DD002B00D18774BDE828
:10843000F0818574FBE700003C010020F806002075
:1084400000040040980200204564BD0100209C40CB
:10845000133B3340E6030020E7030020B404002070
:10846000080A00201C0500202DE9F041384C394E47
:10847000394F207841F23331C2074FF000050CD05C
:10848000A28962B394F90700002800DA4042C0B222
:10849000032829D240F2AE702AE0A570E5732F4A76
:1084A000E571A58192F83830237220F00800A18090
:1084B00040F0020020703D867560B560F560916CFB
:1084C000490005D041F68461A18140F01000207080
:1084D000C0B240F0010020706574BDE8F081658194
:1084E00020F01000207015E0042803D240F651005F
:1084F00060810FE0052802D240F69910F8E740F6B7
:10850000CC42062803D3072801D3082801D2628170
:1085100000E0618197F89D0098B9B088102301B2FE
:10852000B4F90A003622FCF78FF97060F168401A3E
:10853000B1680844B060B6F900104843C013F06059
:108540003886388E10B10120A070C6E7A570C4E748
:10855000100C002078060020980200203C0100202A
:108560002DE9F041554C2678F0077CD05448217A0B
:10857000544D90F8380081427BD0534A2346DFF8AF
:108580004CC1575C93F90E2093F90730874203D012
:108590001CF80170874213D146F002065B1C26705E
:1085A0005BB2E3711CF80110814201D15B1CE371E5
:1085B00094F90710062901DD0621E171521C1CE027
:1085C000434F17F801C0434F844503D017F801C04B
:1085D000844513D126F002065B1E26705BB2E37160
:1085E000795C814201D15B1EE37194F907306FF031
:1085F00005018B4200DAE171521EA273207294F9D8
:1086000007108A1C042A02D941F68462A2812C4AEE
:10861000012912780ADD2B4B56079B6802D543F0DF
:10862000080301E023F00803AB606070B1F1FF3F85
:1086300009DA5107A96802D521F0080101E041F0EB
:108640000801A9606070F9F787FEA078012810D1B1
:1086500021488068A3280CDA94F90700022803DD7A
:108660000220E07105E01EE06FF00101884200DAAF
:10867000E171A089002630B1401E0004000CA081E9
:1086800001D1E671A673E87B04280CD0B5F930104F
:10869000512341220020FCF7D7F82886002802D178
:1086A000E07B10B1A670BDE8F0810C4806700C4864
:1086B0000670207820F001002070F4E7100C0020F4
:1086C0003C01002098020020BC910008C2910008E3
:1086D000CE910008D49100081C0500200C07002052
:1086E000EF060020F23ED03CE13A1F3983370836CE
:1086F000AA34653337321C3113301B2F302E532DE3
:10870000822CBC2B002B4D2AA229000000368E03A0
:1087100000381C07003A1C07003C8808003E880807
:108720000040AA0A0042AA0A0044AA0A0046CC0C49
:108730000048CC0C004A380E004C380E004E380E63
:108740000050380E0052380E0054380E0056380EC5
:108750000058380E005A380E005C380E005E380E95
:108760000060380E0062380E0064380E0066380E65
:108770000068380E006A0000003A2202003C8E03B6
:10878000003EB0050040D2070042AA0A0044CC0CCB
:108790000046EE0E00481111004A3313004C9F149E
:1087A000004E0B16005077170052771700547717BA
:1087B0000056771700587717005A7717005C77171D
:1087C000005E7717006077170062771700647717ED
:1087D0000066771700687717006A7717006C7717BD
:1087E000006E0000003A2202003C8E03003EB005FD
:1087F0000040D2070042AA0A0044CC0C0046EE0E0C
:1088000000481111004A3313004C9F14004E0B1600
:108810000050771700524F1A0054BB1B0056271DFB
:108820000058931E005A0020005C6C21005ED82284
:10883000006044240062B0250064662600661C27A0
:1088400000681C27006A1C27006C1C27006E0000B3
:10885000003400000036000000380000003A00003C
:10886000003C0000003E000000400000004200000C
:10887000004400000046000000480000004A0000DC
:10888000004C0000004E00000050000000520000AC
:10889000005400000056000000580000005A00007C
:1088A000005C0000005E000000600000006200004C
:1088B00000640000006600000068441458585870B6
:1088C000111158585870411158584870111448588F
:1088D00058701411584858701E1500561E15005433
:1088E000A1150052D21500505616004EE916004C44
:1088F0008D17004ABE170048B41800465E1A00449F
:10890000021B0042BC1C0040D91E003EB420003CAB
:108910009F22003AE1220038532300368B24003492
:10892000812500322B2700302028002E5829002CCA
:10893000B02A002A9B2C0028D22D00267C2F002450
:108940002631002202330020FD34001E5C37001C5B
:10895000CC3C001A873E0018BE3F001600400014B1
:1089600000400012004000100040000E0040000CCB
:108970000040000A004000080040000600400004DB
:108980000040000200400000010203040500050051
:10899000010203040104000305020000F0010000CD
:1089A00036010000F8000000BA0000007C00000062
:1089B0007C0000007C0000004114141111144411CB
:1089C000141441110000290052007B00A400CC00C7
:1089D000F5001E01470170019901C201EA0113026D
:1089E0003C0265028E02B602DF020803300359031F
:1089F0008203AA03D303FB0324044C0475049D04DF
:108A0000C504EE0416053E0567058F05B705DF05AD
:108A100007062F0657067F06A706CE06F6061E0790
:108A200046076D079507BC07E4070B08320859088D
:108A30008108A808CF08F6081D0944096A099109A8
:108A4000B809DE09050A2B0A520A780A9E0AC40AE6
:108A5000EA0A100B360B5C0B820BA80BCD0BF30B49
:108A6000180C3E0C630C880CAD0CD20CF70C1C0DD2
:108A7000410D650D8A0DAF0DD30DF70D1C0E400E87
:108A8000640E880EAC0ECF0EF30E170F3A0F5E0F6A
:108A9000810FA40FC70FEA0F0D103010531075107F
:108AA0009810BA10DD10FF102111431165118711C4
:108AB000A911CA11EC110D122E125012711292123C
:108AC000B312D412F41215133613561376139613E9
:108AD000B713D713F61316143614561475149414CA
:108AE000B414D314F214111530154E156D158C15E0
:108AF000AA15C815E7150516231641165F167C162C
:108B00009A16B716D516F2160F172C1749176617AF
:108B10008317A017BC17D917F51711182E184A1864
:108B2000661881189D18B918D418F0180B19261951
:108B300042195D1978199219AD19C819E219FD1970
:108B4000171A311A4C1A661A801A991AB31ACD1AC2
:108B5000E61A001B191B331B4C1B651B7E1B971B46
:108B6000AF1BC81BE11BF91B121C2A1C421C5A1C00
:108B7000721C8A1CA21CBA1CD21CE91C011D181DE7
:108B8000301D471D5E1D751D8C1DA31DBA1DD01DFA
:108B9000E71DFD1D141E2A1E401E571E6D1E831E3E
:108BA000981EAE1EC41EDA1EEF1E051F1A1F2F1FB1
:108BB000451F5A1F6F1F841F991FAE1FC21FD71F4B
:108BC000EC1F002000006400C9002D019201F70194
:108BD0005B02C00224038903ED035204B6041A05A4
:108BE0007F05E3054706AB060F077307D7073B086A
:108BF0009F0802096609C9092D0A900AF30A560B53
:108C0000B90B1C0C7F0CE20C440DA60D090E6B0E6B
:108C1000CD0E2F0F900FF20F5310B41015117611C7
:108C2000D71138129812F8125813B8131814771471
:108C3000D61435159415F3155116B0160E176B177B
:108C4000C91726188318E0183D199919F519511AF2
:108C5000AD1A081B631BBE1B181C731CCD1C261DE4
:108C6000801DD91D321E8A1EE31E3B1F921FEA1F64
:108C700041209820EE2044219A21EF21452299227B
:108C8000EE2242239623E9233C248F24E224342538
:108C90008525D72528267826C82618276827B727A8
:108CA00006285428A228EF283D298929D629222AD6
:108CB0006D2AB82A032B4D2B972BE12B2A2C722CD3
:108CC000BB2C022D4A2D912DD72D1D2E632EA82EA3
:108CD000EC2E302F742FB82FFA2F3D307F30C0305C
:108CE000013141318131C13100323F327D32BA32FE
:108CF000F73234337033AC33E73322345C34953499
:108D0000CE3407353F357735AE35E4351A36503633
:108D10008536B936ED36203753378637B737E937DA
:108D2000193849387938A838D738053932395F3990
:108D30008B39B739E2390D3A373A603A893AB23A63
:108D4000DA3A013B283B4E3B733B983BBD3BE03B53
:108D5000043C263C483C6A3C8B3CAB3CCB3CEA3C6C
:108D6000093D273D443D613D7D3D993DB43DCE3DAE
:108D7000E83D013E1A3E323E493E603E763E8C3E24
:108D8000A13EB53EC93EDC3EEF3E013F123F233FD0
:108D9000333F433F513F603F6E3F7B3F873F933FB1
:108DA0009E3FA93FB33FBC3FC53FCD3FD53FDC3FD2
:108DB000E23FE83FED3FF13FF53FF93FFB3FFD3F2D
:108DC000FF3FFF3FFF3F0000E7382C35002020EF3A
:108DD00020372023332026202100008002000400B9
:108DE0000800100000020004000804000002000453
:108DF00000080010002000400080040000000080F7
:108E000000000040000000200000001000000008EA
:108E100000000004000000020000000100008000CB
:108E200000004000000020000000100000000800CA
:108E300000000400000002000000010000800000AB
:108E400000080140000C0140000C0140000C0140F2
:108E5000000C0140000C0140000C0140000C0140DE
:108E600000100140001001400010014000100140BE
:108E700000100140001001400010014000100140AE
:108E80000014014004080140040C0140040C01409E
:108E9000040C0140040C0140040C0140040C01408E
:108EA000040C014004100140041001400410014072
:108EB000041001400410014004100140041001405E
:108EC000041001400414014008080140080C01404E
:108ED000080C0140080C0140080C0140080C01403E
:108EE000080C0140080C0140081001400810014026
:108EF000081001400810014008100140081001400E
:108F00000810014008100140081401400C080140FD
:108F10000C0C01400C0C01400C0C01400C0C0140ED
:108F20000C0C01400C0C01400C0C01400C100140D9
:108F30000C1001400C1001400C1001400C100140BD
:108F40000C1001400C1001400C1001400C140140A9
:108F500010080140100C0140100C0140100C0140A1
:108F6000100C0140100C0140100C0140100C01408D
:108F7000101001401010014010100140101001406D
:108F8000101001401010014010100140101001405D
:108F9000101401400000000000000000000000006C
:108FA000000000000000000014080140140C014003
:108FB000140C0140140C0140140C0140140C01402D
:108FC000140C0140140C0140141001401410014015
:108FD00014100140141001401410014014100140FD
:108FE000141001401410014014140140000000004E
:108FF0000000000000000000000000000000000071
:10900000FFFFFF0F0FFFFFFFFFF0FFFFFF0FFFFF4F
:10901000FFFFF0FF0FFFFFFFFFF0FFFFFF0FFFFF5E
:10902000FFF0FFFF0FFFFFFFFFF0FFFFFF0FFFFF4E
:10903000FFFFF0FFFFFF0FFFFFFFFFF0FFFFFF0F3E
:10904000FFF0FFFF000000404000000000040000AF
:109050000040000000000400400000000004000088
:109060000040000000040000400000000004000078
:109070000040000000000400000040000000000468
:10908000000000400004000000000080800000009C
:1090900000080000008000000000080080000000C0
:1090A00000080000008000000008000080000000B0
:1090B00000080000008000000000080000008000A0
:1090C00000000008000000800008000000000020F0
:1090D000200000000002000000200000000002004C
:1090E000200000000002000000200000000200003C
:1090F000200000000002000000200000000002002C
:10910000000020000000000200000020000200001B
:109110000000006060000000000600000060000029
:109120000000060060000000000600000060000073
:109130000006000060000000000600000060000063
:109140000000060000006000000000060000006053
:109150000006000000800200040008001000000269
:1091600000040008040000020004000800100020B1
:109170000040008004000000FF7FFFFFFDFFFFFFB5
:10918000FBFFFFFFF7FFFFFFEFFFFFFFFFFDFFFF0D
:10919000FFFBFFFFFFF7FFFFFBFFFFFFFFFDFFFFF1
:1091A000FFFBFFFFFFF7FFFFFFEFFFFFFFDFFFFF0B
:1091B000FFBFFFFFFF7FFFFFFBFFFFFF0102030475
:1091C0000500020304050001030405000102050077
:1091D0000102030404050001020355050010AA1A48
:1091E00055250030AA3A0000AA0A55150020AA2ADF
:1091F0005535FF3F149200080000002020070000B2
:10920000E80600080893000820070020B0090000C5
:109210004863000845020406082D01020304040502
:109220004406070809139D2B1B08B104211355158B
:109230002A40061908019713AD3D1B08D1041ACD29
:1092400004012D17020604050103148020FF8BAAD8
:109250000A02019C15AA0A551500085920AA2A5588
:1092600035FF3F072903010504060203127C15732D
:10927000FFFF04FF8080010125025B6402130A13D3
:10928000B56612081201100C050406020301010361
:10929000070505280B010203040206070303040C5B
:1092A0003D0706040509191F191904310506062F83
:1092B000AA1A381EAA1A064902290C2902312E4080
:1092C000FD3969260211042F405F020C26405B26FF
:1092D0002ACD55155515123902017F0316D0071AEC
:1092E000FF01013B0261AA6C080108A80916C4919C
:1092F000220312100A17401C12600A16901B014923
:0893000013C966020008000019
:020000040800F2
:10FC00004A46545A594D46312D4E3330202020203B
:10FC1000050406020301AA0AAA0AAA0AAA0AAA0A4B
:10FC2000AA0ADE3F00100000FF0131000201664613
:10FC300000400040513800400040004000400101B9
:10FC400000400040FF387B257B257B25FF003333B8
:10FC50000201401F00016626B81E6626FFFFFFFF57
:10FC6000FFFF01010100010000000300000202008B
:04FC70000000AA5591
:04000005080000ED02
:00000001FF
